:100000000C949F040C94BC040C94BC040C94BC048D
:100010000C94B3140C94BC040C94BC040C94BC0459
:100020000C94BC040C94F1050C94BC040C9485064F
:100030000C94BC040C94BC040C94BC040C94BC0440
:100040000C94BC040C94BC040C94BC040C94BC0430
:100050000C94BC040C94BC040C94BC040C94BC0420
:100060000C94BC040C94BC04DC0B1A0C2D0C5A111F
:100070005A115A115A115A115A115A115A115A1128
:100080005A115A115A115A115A115A115A115A1118
:100090005A115A115A115A115A115A11320C5A1135
:1000A0005A0C6E0C890CB10CDF0CF00C040D2E0DEB
:1000B0005A0D5A0D620E620E620E620ED90B9F0E21
:1000C000630D7A0D820F8C0F0D100D100D100D1099
:1000D0000D105A115A115A115A115A115A115A1116
:1000E0005A11A10FF70F0D106364696E6F7073756D
:1000F00078585B003C656D7074793E20202020208C
:10010000006572726F723A20777269746520616659
:1001100074657220666F726D61740053494F2D458E
:1001200072726F723A2025690053494F3A434D4429
:100130002054696D656F75740053796E6320576143
:1001400069742E2E2E2020200053746F7070656409
:100150002E2E2E202020003E4E65773C2020202091
:10016000202020004572726F7220696E69742046EB
:1001700041543A20257500252E30386C7820252EE4
:1001800030386C78004572726F7220696E69742025
:1001900053443A202575005344524956452E415444
:1001A00052206E6F7420666F756E6400252E327853
:1001B00020252E327820252E327820252E327820C8
:1001C0002563202575006572726F723A206372652F
:1001D000617465206E65772066696C65000F111388
:1001E00015181A1C1E212325325344726976653175
:1001F00033203230323231323034206279204B4277
:1002000072006279204B42722056312E33005344E3
:10021000726976652D4D41580053444D58252E3452
:10022000750053444D58256875004154520054469A
:10023000542D49443A20252E30347800546170659D
:100240002D456D750058313A2025692C2058323AD9
:100250002025692C2059313A2025692C2059323A21
:100260002025690020202020202020202020202060
:100270000025692066696C65732C207061676520B4
:1002800025692F256920202573202020202020206B
:10029000202020202000C50100000000F0001801EF
:1002A00059CE0000FFFF1E01152059010F00A500C7
:1002B00050001E0059CE0000FFFF22016C205F019C
:1002C0000F00CD0050001E0059CE0000FFFF21019D
:1002D000CE2365019000A50050001E0059CE0000FD
:1002E000FFFF2001B3236B019000CD0050001E00E2
:1002F00059CE0000FFFF1F01152070010F002D00D7
:100300005A001E0059CE00001F052A01EC23770178
:100310000F0055005A001E0059CE00001F0529018C
:10032000EC237E010F007D005A001E0059CE000014
:100330001F052801EC2385010F00A50046001E00C3
:1003400059CE00001F052701EC238A010F00CD00C4
:1003500050001E0059CE00001F052601EC2390011D
:100360000F00F5005A001E0059CE00001F052501A0
:10037000EC239701A4007D003C001E0059CE000034
:10038000FFFF24019D276B01A400A5003C001E0077
:1003900059CE0000FFFF230115209C01A4002D0071
:1003A0003C001E0059CE0000FFFF31019221A00148
:1003B000A40055003C001E0059CE0000FFFF300194
:1003C0008121A501A4007D003C001E0059CE000043
:1003D000FFFF2F0134206B01A400A5003C001E008C
:1003E00059CE0000FFFF2E011520A801A400CD006A
:1003F0003C001E0059CE0000FFFF2D019D20AD01E5
:10040000A400F5003C001E0059CE0000FFFF2C01A7
:100410009B21C5010F002D009600F00059CE000071
:10042000FFFF2B01A226B2010A00C80032001E0005
:1004300059CE000000003A01FA1FB6010A00280058
:10044000DB001E0059CE0000000039016F20C601FC
:100450000A005000DB001E0059CE000000003801E9
:100460006F20D6010A007800DB001E0059CE000084
:10047000000037016F20E6010A00A000DB001E002B
:1004800059CE0000000036016F20F6015000C80070
:1004900050001E0059CE0000000035010420FC0170
:1004A000B300C80032001E0059CE0000E00734013E
:1004B0006C2000020A00F00032001E0058540000B8
:1004C000DFFF33016C200402B300F00032001E0095
:1004D00059CE00001F0032015E20C5010A0018013C
:1004E000E5003F01000000000000220234264154D4
:1004F00052415458434153434F4D42494E4558454C
:10050000584558584644544150494D47424153522A
:10051000454144590000002421E318C318E318049E
:100520002104210000000000000000000000000085
:1005300000000000000421821041084108410861C8
:100540000861084569456982108210A210A210C393
:1005500018042100008210410820002000200041E2
:100560000841084569456941084108610841086139
:1005700008821000008210200020002000200020AF
:100580000041084569456941084108410841084161
:10059000086108A2108210200020002000200041E5
:1005A0000861086108610861086108610861084123
:1005B000086108A210A21041082000200041086133
:1005C000088210FFFFFFFF0000A210A2108210613E
:1005D000088210A210C318610841084108821082E5
:1005E00010FFFF1F001F00FFFF0000E318A2108292
:1005F000108210C318E3188210610861088210FF8E
:10060000FF1F001F001F001F00FFFFC318A2108262
:10061000108210C318E318821082108210A210FFFB
:10062000FF1F001F001F001F00FFFFC318A2106163
:10063000088210C318C318821061088210A210E348
:1006400018FFFF1F001F00FFFF0000A210821061B3
:10065000086108A2108210610841088210C31804C2
:10066000212421FFFFFFFF0000C318A210821041C8
:1006700008610882101F000000200041088210C39A
:1006800018E318E318E318C318C318A2106108612F
:10069000086108610800000000200041086108A20C
:1006A00010C318C318A210A210A210821061084132
:1006B00008610882106108000020002000610882A3
:1006C00010A210A2108210821082106108610861CD
:1006D000088210A210C3186108410841086108820D
:1006E00010A210A21082108210821082108210823A
:1006F00010C318000000000000000000000000000F
:1007000000000000000000000000000000000000E9
:10071000000000000000000000000000005F00007A
:100720000007000700147F147F14242A7F2A122355
:100730001308646236495522500005030000001C6E
:100740002241000041221C0014083E081408083E03
:100750000808005030000008080808080060600021
:100760000020100804023E5149453E00427F4000EF
:1007700042615149462141454B311814127F1027DF
:10078000454545393C4A4949300171090503364917
:10079000494936064949291E0036360000005636BA
:1007A00000000814224100141414141400412214EF
:1007B000080201510906324979413E7E1111117E2C
:1007C0007F494949363E414141227F4141221C7FB8
:1007D000494949417F090909013E4149497A7F0850
:1007E00008087F00417F41002040413F017F0814FD
:1007F00022417F404040407F020C027F7F0408106E
:100800007F3E4141413E7F090909063E4151215E3B
:100810007F09192946464949493101017F01013FB4
:100820004040403F1F2040201F3F4038403F63145E
:1008300008146307087008076151494543007F4168
:10084000410002040810200041417F00040201021F
:1008500004404040404000010204002054545478B9
:100860007F484444383844444420384444487F381E
:1008700054545418087E09010218A4A4A47C7F08CB
:1008800004047800447D40004080887A007F10286E
:10089000440000417F40007C041804787C08040474
:1008A000783844444438FC2424241818242418FCA0
:1008B0007C080404084854545420043F4440203C1D
:1008C0004040207C1C2040201C3C4030403C4428C0
:1008D0001028441CA0A0A07C4464544C440008365A
:1008E000410000007F000000413608001008081099
:1008F000087846414678FFFFFFFFFF426C6F636B4D
:10090000202575202020202000426175643A202592
:1009100075204C656E6774683A20257520476170B4
:100920003A2025752020202000456E6420200042BA
:100930006C6F636B202575202F20257520001124F6
:100940001FBECFEFD8E0DEBFCDBF12E0A0E0B1E028
:10095000ECE7FBE702C005900D92A830B107D9F78C
:1009600026E0A8E0B2E001C01D92A33EB207E1F785
:100970000E946F110C94BC3D0C9400000F931F93C8
:1009800090912102911131C0E0914001F09141011B
:100990002281338194E1899F200D311D1124F901B9
:1009A0007096A591B4918C9182FF03C00FE110E085
:1009B00002C009E51EEC462FF9013296849190E0C1
:1009C00032962491622F70E06B5F7F4F0596413025
:1009D00029F0423029F400E018EF02C000EE17E0E1
:1009E00021E043E050E00E94AC2A1F910F9108954E
:1009F000CF93DF9340E050E090E060E3680F71E355
:100A0000E0914001F09141010280F381E02D9F01CE
:100A1000240F351FF9017096C591D491F901A59164
:100A2000B49128812B7F2883891302C024602883F6
:100A300020E3290F11962C931197823048F08913E7
:100A400003C011967C9304C0913011F411966C93FD
:100A50009F5F4C5E5F4F953099F680912102811126
:100A600002C00E941623DF91CF910895A0E1B0E06B
:100A7000ECE3F5E00C94D2346B017C018E010F5F46
:100A80001F4F80E1F80111928A95E9F7C701B6017D
:100A9000605F7F4F8F4F9F4F0E94741E61157105DD
:100AA0008105910569F126E932E03A8329834601FF
:100AB000570124E0B694A794979487942A95D1F788
:100AC0009C828B82F1E0CF16F8E0DF06F2E0EF06C1
:100AD000F10418F020E031E002C020E830E03E836D
:100AE0002D830E94D91680E1F801A4EBB2E00190B9
:100AF0000D928A95E1F780E00E94991680E005C08A
:100B000086EC91E00E94A42581E06096ECE00C94D4
:100B1000EE34E62FF0E0EC54FB4F6AE00E94203404
:100B200080638083906391830895E4EBF4E08C54B8
:100B30009B4F1192E817F907E1F708959091B505D9
:100B40009F939091B4059F931F928F93ECEDF5E0E6
:100B500083811F928F9382811F928F9381811F9235
:100B60008F9380811F928F938CEA91E09F938F9354
:100B700088EC95E09F938F930E948D3788EC95E0E9
:100B80000E947A268DB79EB740960FB6F8949EBF06
:100B90000FBE8DBF089580E090E00E948629E0E7B7
:100BA000F0E0808181608083E1EBF0E0808187600C
:100BB00080830895E0E7F0E080818E7F808310924B
:100BC000B10080912102E0914001F091410195E056
:100BD000899FE00DF11D11240190F081E02D099510
:100BE00008951F920F920FB60F921124EF92FF9269
:100BF0000F931F932F933F934F935F936F937F9325
:100C00008F939F93AF93BF93CF93DF93EF93FF9314
:100C1000809108028F5F809308028F7309F50E940C
:100C20005F37EC010E945F378C0180E090E00E940A
:100C30008629C8016CE271E00E944034FC01CE01BB
:100C400068E770E00E9440342EE0E22E22E0F22EAF
:100C500000E010E028E03CEF42E0BF010E94FC2BE6
:100C6000FF91EF91DF91CF91BF91AF919F918F91C4
:100C70007F916F915F914F913F912F911F910F91B4
:100C8000FF90EF900F900FBE0F901F9018950F934D
:100C90001F9380910D0281111EC0E091BE05F0915D
:100CA000BF05868981FF09C02FE781E397E12150C5
:100CB00080409040E1F700C000008BE0809381000D
:100CC00000EE17E021E043E050E065E070E085E0F1
:100CD00090E00E94AC2A81E080930D021F910F9159
:100CE00008950F931F931092810010920D0200E05F
:100CF00010E021E043E050E065E070E085E090E046
:100D00000E94AC2A1F910F9108951F920F920FB667
:100D10000F9211242F933F934F935F936F937F9381
:100D20008F939F93AF93BF93EF93FF9380910D02A7
:100D3000882319F08F5F80930D0280910D02853119
:100D400010F00E947106FF91EF91BF91AF919F91BA
:100D50008F917F916F915F914F913F912F910F9064
:100D60000FBE0F901F901895A0E0B0E0EAEBF6E000
:100D70000C94D7348CE392E09093BF058093BE052A
:100D80008091380290913902A0913A02B0913B02D1
:100D90008093400290934102A0934202B093430299
:100DA000E12CF12C60E0C7010E949018882309F41F
:100DB0005CC004EB14E0C1E6D0E0F801D1908F01F3
:100DC000CE010E94743DD8124CC02196F4E00F3B36
:100DD0001F0799F7E091BE05F091BF0580819181D1
:100DE000A281B38180879187A287B38714861586F5
:100DF0001686178620E130E040E050E0BA0180E03E
:100E00000E94981AC091BE05D091BF0581E08E8BDB
:100E10009091B8048091B904892B813011F481E25A
:100E20008E8B8A899B89AC89BD89BC01CD016051BB
:100E30007109810991091E8915FD05C020E830E07E
:100E400040E050E004C020E031E040E050E00E948B
:100E50005434213D32404105510580F010681E8B0D
:100E60000DC0EFEFEE1AFE0A9DCFE091BE05F091A6
:100E7000BF05168A87E991E00E94A425CDB7DEB7A9
:100E8000E7E00C94F334A7E0B0E0E9E4F7E00C9479
:100E9000CC348091DD05811155C040E064E070E004
:100EA0008CED95E00E94471F823031F489E291E099
:100EB0000E94A4250C946B11AFE7BCE01197F1F7E9
:100EC00000C00000359BFECF882309F43BC0909101
:100ED0000F029923B1F01F928F938BE191E09F93C2
:100EE0008F9384EB94E09F938F930E948D3784EBD4
:100EF00094E00E947A260F900F900F900F900F9021
:100F00000F908091C205883239F081E09091C1053F
:100F1000911180E08093C1058091C105882361F023
:100F2000E091C205EB3018F0E8EEF1E003C0F0E02C
:100F3000E352FE4F849101C088E690E00E94131FA7
:100F40000C946B111091DD058091DC059FEC980FDE
:100F5000943080F42091C005813319F42093B605B4
:100F60001AC090E030E0205D3F4F8217930771F484
:100F700081E00FC0813711F00C946B1180EB810F71
:100F8000843008F0FAC380E38093DC058091DC05AF
:100F90008F708093B6058091B605482F50E0B8E178
:100FA0008B9FF0011124E45CFD4FF093BF05E093AB
:100FB000BE059689292F297011F40C946B111335F5
:100FC00009F40AC1292F2B7F268B123209F4DCC0C9
:100FD00018F4113241F000C1103509F4F9C0173589
:100FE00009F4F6C0F9C08091BD05813019F4009173
:100FF000E70501C000E093FF29C081E40E942C1F97
:1010000062E08091B6050E94BE040E94470600235C
:10101000C1F08091E505811105C060E87EEC82E0B9
:1010200090E0C2C0813041F0E091BE05F091BF0573
:1010300086898460868BEDC060E87EE985E090E07B
:10104000B3C060E078E681E090E0AEC094FF07C0F6
:10105000C12C78E6D72EEE24E394F12C07C060E192
:10106000C62E68E6D62EEE24E394F12C8330E1F20E
:10107000811111C088E1849FF001859FF00D11243A
:10108000E45CFD4F82899389A489B589C816D90685
:10109000EA06FB0649F6011103C000E810E002C0B1
:1010A00000E011E01092BD05E091BE05F091BF0592
:1010B000878980FDB9CF868986FDB6CF83FF03C0BF
:1010C000877F868B08C081E40E942C1F62E080919C
:1010D000B6050E94BE0480E091E00E949505E09173
:1010E000BE05F091BF05868984FF04C0812C912C38
:1010F00054011CC050E1852E912CA12CB12C16C09E
:10110000E1E0CE16DE06E104F10420F0C12CD12C82
:101110007601D3949601B501A40181E00E94981A4A
:10112000892B99F08C0C9D1CAE1CBF1CE091BE0558
:10113000F091BF05C288D388E488F588C818D9081B
:10114000EA08FB08E9F680E001C081E0E4EBF4E0A6
:1011500098012C543B4F9FEF9193E217F307E1F76F
:10116000882379F01092B4041092B504E091BE0582
:10117000F091BF0586898460868B81E091E00E94B2
:10118000A42540E0B801D8C693FF1FC081E40E94A7
:101190002C1F62E08091B6050E94BE040E944706A3
:1011A00060E078E082E090E00E94360581113CCF5B
:1011B0001091B605E091BE05F091BF058089918937
:1011C0009093DF058093DE054AC727FF2DCF65CFBB
:1011D00062E00E94BE0426C061E00E94BE048091CD
:1011E000DD059EEA980F923050F4E091BE05F09133
:1011F000BF05968993FF16C0833529F413C08E343A
:1012000089F08F3479F08F3321F48091C2058832D0
:1012100049F480910F02882309F4C6C38EE40E942A
:101220009E05C2C381E40E942C1F8091700080FD46
:101230000E94DA058091DD05803509F408C158F473
:101240008E34B1F008F0A0C08F3311F00C946B1104
:101250008091C20529C3833509F45DC2873509F43D
:10126000F6C0823511F00C946B110E944706EFC056
:10127000E090BE05F090BF05D70152964D905D906D
:101280006D907C90559756968C9183FF0BC09091F2
:10129000BD05913009F472C0412C38E6532E662406
:1012A0006394712CB82FB074BD8385FF03C000E038
:1012B00011E002C000E810E0C12EDD2480E090E0E3
:1012C00053014201E0E88E2221EE35E03C832B837E
:1012D0001C013CE0230E311CDC011196BF83AE8360
:1012E0000E94743DEB81FC818193FC83EB838E81B2
:1012F0009F812816390681F7FD81F11113C0809175
:10130000E9059091EA05A091EB05B091EC058815EF
:101310009905AA05BB0531F48091E70590E08C158D
:101320009D0561F1C1012091E105213069F6C0926E
:10133000E7050093E8052D81222341F03DE2430EAD
:1013400034EB531E611C711C0DE710E0D70156965B
:101350008C9185FF06C0B0E84B0EB1E05B1E611CAE
:10136000711C980140E050E0C301B2010E94543466
:101370003093E3052093E4054093E50540E06CE0FD
:1013800070E081EE95E0DAC56CE070E081EE95E00A
:101390000E948E1F81119FC70091BE051091BF054D
:1013A000D8015696EC915697F091E705E3FF09C0F6
:1013B000FF2311F0E06202C0EF7DD8015696EC9356
:1013C00042C02091E505822F90E0A0E0B0E09C01B2
:1013D000AD012F5F3F4F4F4F5F4FA091E105B0E050
:1013E0000E94B9349B01AC01A091E305B0E0BA2F93
:1013F000AA278091E405A80FB11D0E94C4349B0167
:10140000AC01AF2FB0E0BA2FAA278091E805A80F52
:10141000B11D0E94C434E4FD04C0605F7F4F8F4F54
:101420009F4FE5FF04C06058714081099109F801A0
:101430000289138924893589601771078207930708
:1014400011F083E001C081E08093BD0523C780E8EF
:1014500090E09A8389831092BD05C090DE05D090FC
:10146000DF05C114D10409F452C1E091BE05F09129
:10147000BF05E689E6FD73C0E1FF15C090910E023D
:101480008091B605981731F00E944B2F8091B605D8
:1014900080930E0242E051E0BE016F5F7F4FC601B4
:1014A0000E94C52F3DC0F4E0CF16D10458F421E0CE
:1014B000C21AD108D694DC2CCC24D794C794E12C42
:1014C000F12C1CC0E5FF03C0A0E0B1E002C0A0E821
:1014D000B0E0BA83A983A60160E070E09A01AB0195
:1014E00024503109410951090E94B9346B017C0132
:1014F00030E8C30E31E0D31EE11CF11CE4FD05C051
:1015000080E1C80ED11CE11CF11C8091DD05298110
:101510003A81823549F4B701A60180E00E94981A09
:10152000892B09F4F4C0F0C0B90184EB94E00E9467
:101530008E1F8111D0C60E944706E091BE05F09132
:10154000BF05878980FDE3C029813A81B701A601E3
:1015500081E00E94981A892B09F4D9C09BC680911A
:10156000DD05823551F060E870E084EB94E00E9484
:101570008E1F882309F4CBC0AEC680E890E00E949D
:10158000950594E0C916D104F0F0E090BE05F09006
:10159000BF05F70182899389A489B589BC01CD0172
:1015A00064587F4F8F4F9F4F2DE730E040E050E071
:1015B0000E94543449015A018901F8E6CF16F1E03E
:1015C000DF0629F574C0C6019695982F8827979550
:1015D0008795835190402091C30577E0972E920E16
:1015E00004EB14E07C0120E8E20EF11C5C013FEF0B
:1015F000A31AB30A0E94743D873009F4892DD801DB
:101600008D938D01C501AE14BF0481F7BECFB9E63D
:10161000CB16B1E0DB0609F04FC060E0F70180892E
:1016200091890E949018A4EBB4E080E090E030E251
:101630002D914FEB420F4A3120F040ED420F4A30DE
:1016400030F4E82FF0E0EC54FB4F20838F5F9730AD
:1016500011F09A3049F4981738F0E82FF0E0EC5484
:10166000FB4F30838F5FF7CF9F5F9B3009F7EFEB26
:10167000F4E08291858324E0E43BF207D1F7E4ECC7
:10168000F4E084E395E08E179F0711F01192FBCFF1
:10169000003932E0130710F086E401C082E4809341
:1016A000B40481E791E09093B8048093B7049092DA
:1016B000B6048092B50424C081E7C81681E0D8063C
:1016C000F8F09601ADE7B0E00E94A334AB01BC0195
:1016D0004D52544B610971092DE730E080E00E94C2
:1016E000981A8D37910520F096012F5F3F4F02C069
:1016F00020E030E0309331052093320580933305AC
:1017000080E890E09A83898369817A8114C4698131
:101710007A8141E011C490910D02911190E1909372
:10172000B404E091BE05F091BF05868987FF03C030
:1017300090689093B40485FF05C09091B4049062C2
:101740009093B40482FF07C09091B4049460909386
:10175000B4048B7F868B878980FF05C08091B40499
:1017600088608093B404809102018093B50480EE78
:101770008093B6041092B704ADC081E40E942C1F80
:10178000E091DD05EB3D09F48AC01F7088EF95E01C
:101790009093BF058093BE058E2F90E0FC01E05C26
:1017A000F109E034F10508F085C5EC5CFF4F0C94BD
:1017B000953400E010E0B2C280E091E00E9495050F
:1017C0008091DE059091DF0500EC14E06C01A5E14D
:1017D000CA0ED11C7C01BFEFEB1AFB0A60E00E942D
:1017E00090188823D9F0EC14FD0429F48091B404F6
:1017F000F801808313C0A4EBB4E0C8010B96F80194
:101800002D912193E817F907D9F78091B805D801F0
:101810001B968C93045F1F4FC701DCCFE4EBF4E011
:1018200084858193B5E0E53AFB07D1F740E061EFAD
:1018300070E082C38091DE058A3F08F03BC580934B
:10184000C2051092C105EFE7FCE03197F1F700C047
:10185000000083E40E942C1F5FCB8091DE05809303
:10186000C30518C583E292E0A4EBB4E04DEC54E06C
:10187000FC012191CF012D93F4E0AD3CBF07C1F7EE
:10188000A8EFB5E085EE94E02D91FA012193AF0128
:101890008E179F07C9F740E061E370E04DC3E09108
:1018A000BE05F091BF0586898093B40440E061E0F5
:1018B00070E042C36091DE057091DF0580E090E04A
:1018C0000E940B176093B4047093B5048093B60420
:1018D0009093B70440E064E070E02EC364E070E0F1
:1018E00084EB94E00E948E1F8111F5C46091B404D2
:1018F0007091B5048091B6049091B7046093C405CB
:101900007093C5058093C6059093C7050E94D916AC
:10191000C1C46091C4057091C5058091C6059091C0
:10192000C7050E94D9168FE79CE00197F1F700C028
:10193000000083E40E942C1FAFE7BCE01197F1F791
:1019400000C0000060E072E084EB92E00E94041F9F
:10195000182F60E072E084EB92E00E94331F812F29
:10196000B8C46091C4057091C5058091C605909179
:10197000C7050E94D91640E260E072E084EB92E075
:101980000E94471FEFE9FFE03197F1F700C0000028
:10199000882361F06091C4057091C5058091C605EA
:1019A0009091C7050E94D9168EE493C481E40E94E9
:1019B0002C1F80E00E94991681117CC46BC4609139
:1019C000DE05662309F466C4E9EEF1E0A4EBB4E0B9
:1019D00080E094919D938F5F31966813FACFAAC2ED
:1019E0000E94D0168091DE05882319F00E94B4066B
:1019F0005FC48FE79CE00197F1F700C0000083E42B
:101A00000E942C1F0C9400009091DE05953008F088
:101A100051C4A8E19A9FF0011124E45CFD4F86892E
:101A200083FD02C08E7F01C0867F868BE0914001DE
:101A3000F09141010280F381E02DB4E19B9FE00D24
:101A4000F11D1124859194914CE050E064EF70E019
:101A500003960E946F378091C0055BC2E091DE055E
:101A6000E53008F027C428E1E29FF0011124E45C8E
:101A7000FD4F868980FD08C08EE090E00E949505AC
:101A800040E06EE070E058C2F093BF05E093BE0501
:101A900084819581A681B7818093FC059093FD0593
:101AA000A093FE05B093FF05908981899093DE0590
:101AB0008093DF0560E08091DE059091DF050E9454
:101AC0009018082F3CC06BE070E08DEE95E00E940E
:101AD0008E1F811100C48091DF05882309F4DAC3C9
:101AE0001091DE05812F806F8093DD051092DF0558
:101AF0001092DE05E090DE05F090DF058091DD05B7
:101B0000803F08F0B5C160E0C7010E9490188823AB
:101B100009F4F2C1EDEEF5E0A4EBB4E0819181119E
:101B2000C1C1119635E0E83FF307C1F78091DD05AB
:101B3000803F08F0BCC183EE8093DD0501E0209179
:101B4000B8052093BF048091DD05833E61F4E091E8
:101B5000BE05F091BF05808991899093C10480935F
:101B6000C0041EE0A7C0853E09F0A3C0A091BE0539
:101B7000B091BF0552964D915D916D917C915597B5
:101B80004093C0045093C1046093C2047093C30493
:101B90008091B905D090BA058093C404D092C50451
:101BA0008091BB059091BC059093C7048093C604B7
:101BB000E8ECF4E086EE94E030E231938E179F0774
:101BC000E1F752966D917D918D919C915597287179
:101BD00019F420E32093D10444EBE42E44E0F42EE6
:101BE0001AE05AE0852E912CA12CB12C61157105BB
:101BF0008105910551F0A50194010E945434606360
:101C0000D7015D966C93B901CA011150B1E0EB1A8E
:101C1000F1081111EBCF8DE28093D7048093DA04A1
:101C20008AE38093E0048093E3048D2D869590E011
:101C30008454984F64E670E00E942C34962F182F3D
:101C40006FE1892F0E94890561E2812F0E94890539
:101C50008091B9059091BA0525E0969587952A95CA
:101C6000E1F764E28F700E9489058091B90567E20F
:101C70008F710E9489058091BC056AE286958695E0
:101C800086950E9489058091BB059091BC0535E041
:101C9000969587953A95E1F76DE28F730E948905D5
:101CA0008091BB058F7160E3880F0E94890512E364
:101CB00001C01CE0011104C082E390E00E94950580
:101CC000612F38C161E08091DE059091DF050E94AF
:101CD0009018811106C080E090E0FC01EC54FB4FAD
:101CE00009C0E4EBF4E080E090E00196219121113D
:101CF000FCCFF3CFCF01845B94408F3F910509F077
:101D000010F41192F7CF8091DD05865E60E071E0FE
:101D100002C0759567958A95E2F70DC160E0C8012C
:101D20000E949018882319F00F5F1F4FF7CF109370
:101D3000B5040093B40440E062E070E0FDC080911F
:101D4000DE058150843118F084E18093DE05009136
:101D5000DE058090FC059090FD05A090FE05B090FA
:101D6000FF0510E08FE2D82E60E080E090E00E9456
:101D70009018E091BE05F091BF05882309F450C08A
:101D80008091B80584FF4CC08091B4048E3209F074
:101D900047C08091B5048E3209F042C0011107C0DE
:101DA000A12FB0E0AC54BB4F8FE38C9339C00150EE
:101DB000448055806680778080819181A281B38143
:101DC00084839583A683B783E12CF12C60E0C7015F
:101DD0000E949018882341F2E091BE05F091BF0562
:101DE00080819181A281B381481659066A067B06DB
:101DF00099F41C50E12FF0E0DF01AC54BB4FDC92B2
:101E0000A4EBB4E0EB54FB4FCF010B962D91219343
:101E10008E179F07D9F7A8CFEFEFEE1AFE0AD6CF9D
:101E200084829582A682B782812F90E0DC01AC5437
:101E3000BB4F119520E03D91E22FF0E0EC54FB4FB9
:101E400030832F5F2113F7CF8195811103C010924A
:101E5000B40481E0E82FF0E0EC54FB4F10828F5F78
:101E6000C9F76091DE05FCE06F9FB001112463C0EB
:101E7000153008F048CE28E1129FF0011124E45CEF
:101E8000FD4FF093BF05E093BE058091FC05909156
:101E9000FD05A091FE05B091FF0584839583A6837F
:101EA000B78331CE9C91891709F43BCE21C0153000
:101EB000D0F488E1189FF0011124E45CFD4FF09309
:101EC000BF05E093BE058091FC059091FD05A091B2
:101ED000FE05B091FF0584839583A683B78360E0F8
:101EE000C7010E949018F092DF05E092DE05B7C0AE
:101EF0009FEFE91AF90A07CE8091DD05803F08F0CF
:101F0000D9C1BACD8091DE05853008F081E080939B
:101F1000C0050E94F804BEC16091DE05E091DF05B6
:101F2000F0E0E054FA4FA4EBB4E0862F91919D933A
:101F30008150E1F770E040E084EB94E00E94C41F20
:101F4000CAC160E080E090E00E949018811116C044
:101F50008091DE05882309F49DC1E091BE05F091D2
:101F6000BF058091380290913902A0913A02B09158
:101F70003B0284839583A683B7837ECD8091B80589
:101F800084FFE6CF8091B4048E3211F78091B504BE
:101F90008E32F1F6E091BE05F091BF05C480D58088
:101FA000E680F78080819181A281B38184839583CB
:101FB000A683B7838091DE05882351F200E010E00C
:101FC00060E0C8010E949018882311F2E091BE05DC
:101FD000F091BF0580819181A281B381C816D90695
:101FE000EA06FB0609F4A7CD0F5F1F4FE9CF8091EA
:101FF000380290913902A0913A02B0913B0280934D
:10200000FC059093FD05A093FE05B093FF0560E0ED
:1020100080E090E00E9490183DC11530B0F4A8E136
:102020001A9FF0011124E45CFD4FF093BF05E0938B
:10203000BE058091FC059091FD05A091FE05B09133
:10204000FF0584839583A683B78360E08091DE05D6
:102050009091DF050E949018882309F42BC190917C
:10206000B805E091BE05F091BF0594FF09C08081DD
:102070009181A281B38184839583A683B78301C1B3
:102080004081518162817381408751876287738764
:10209000148615861686178686898870868B90FD2D
:1020A00002C0178A02C081E0878B8091BC04813412
:1020B00009F049C08091BD04843509F0B1C0809118
:1020C000BE04823509F0A1C020E130E040E050E0DC
:1020D000BA0180E00E94981AE090BE05F090BF051A
:1020E000F7018689982F9160968B2091B804909182
:1020F000B904922B913011F48162868BF7018289A9
:102100009389A489B589BC01CD0160517109810908
:102110009109D688D5FE05C020E031E040E050E0CE
:1021200004C020E830E040E050E00E945434213DFB
:1021300032404105510508F47AC08D2D8068D701E1
:1021400056968C9374C0883559F48091BD048634BA
:1021500009F066C08091BE04843409F061C01AC0E1
:10216000833459F48091BD04813409F059C08091C1
:10217000BE04833509F054C00DC0823409F050C04C
:102180008091BD04893409F04BC08091BE048E3427
:1021900009F046C024E030E040E050E0BA0180E0C1
:1021A0000E94981A8091B404863469F48091B50431
:1021B000853579F48091B6048A3459F48091B70456
:1021C000893439F42DC08F3F21F48091B5048F3FBD
:1021D00039F1E091BE05F091BF058689982F916194
:1021E000968B42895389648975894130B8E65B07CB
:1021F000B1E06B077105D8F041305840624071057D
:1022000010F4816913C0816311C0883549F40E94BC
:102210004B2FE091BE05F091BF058689836006C013
:10222000E091BE05F091BF058689816C868B8FEFAA
:10223000810F843030F560E08091DE059091DF05FC
:102240000E94901884EB94E00E949220E09140015B
:10225000F09141010280F381E02D34E1139FE00D04
:10226000F11D1124859194914CE050E064EB74E0F1
:1022700003960E947E3780912102811102C00E9444
:102280001623E091BE05F091BF05868983FF02C049
:102290000C944B0880910F02882321F083E40E9464
:1022A0009E0506C08FE79CE00197F1F700C0000093
:1022B00083E40FC080910F02882321F085E40E94FF
:1022C0009E0506C0AFE7BCE01197F1F700C0000023
:1022D00085E40E942C1F2796E2E10C94E834A4E0E8
:1022E000B0E0E5E7F1E10C94CC34459A3D9882E00A
:1022F0008093680080E280936C0080B7846880BF20
:102300008FE080937E0083B5816083BD84E79BEC82
:10231000909389008093880080916F008260809301
:102320006F001092C1051092C3051092C005109263
:10233000B6051092BD0580E690E00E94743D809342
:10234000C2050E945027E0914001F09141010190A7
:10235000F081E02D099580913F0182FF03C081E06B
:102360008093C00588E690E00E94131F61E0809191
:10237000B6050E94BE040E942B152FEF31EE44E0FB
:10238000215030404040E1F700C000000E9471152C
:102390008823E1F11F928F9385E891E09F938F93BB
:1023A00084EB94E09F938F930E948D3784EB94E0AD
:1023B0000E947A268091BB028F938091BA028F93FC
:1023C0008091B9028F938091B8028F938091B70268
:1023D0008F938091B6028F938091B5028F938091F5
:1023E000B4028F9387E791E09F938F9324EB34E0BF
:1023F0003F932F930E948D3784EB94E00E947A26BE
:102400000FB6F894DEBF0FBECDBF7AC08DB5816028
:102410008DBD8CB58D7F8CBD8CB58E7F8CBD1092A3
:10242000520210926A021092820210929A02109244
:10243000B2020E943D178823B9F01F928F9384E661
:1024400091E09F938F9384EB94E09F938F930E94EE
:102450008D3784EB94E00E947A260F900F900F90B6
:102460000F900F900F904CC089E08093210266E995
:10247000E62E61E0F62E91E09B83C7010E947C3D31
:102480006093FC057093FD058093FE059093FF0516
:102490006F3F7F4F8F4F9F4F89F0C70104960E9477
:1024A000823D9093DF058093DE058B81806F809362
:1024B000DD05F1E7F093DC050E9443072B812F5FD8
:1024C0002B8336E0E30EF11C2530B9F61092210281
:1024D0000E9416238091380290913902A0913A020D
:1024E000B0913B028093FC059093FD05A093FE05FF
:1024F000B093FF050E94B4068091C0050E94F804C5
:1025000060E08091B6050E94BE047894612C712C25
:1025100044EB54E05C834B83212C312C210158E1A6
:10252000852E0E94C82D882309F45AC1809170001D
:1025300080FF03C00E94DA053EC10E942528009753
:1025400009F446C110922406FC017096259134913D
:102550003C832B833A832983FC01C590D490760178
:10256000F89448EF55E05093BF054093BE05209185
:102570002102211116C0F6012081243491F4E0914A
:102580004001F091410122813381AC01421B530B88
:102590009A0135952795359527955DEC259F902CCB
:1025A0001124FC01729625913491F90109958C0151
:1025B00078948091C005981679F0EB81FC81808138
:1025C00082FF0AC09092C005911002C00E94B4061A
:1025D0008091C0050E94F804F60180818E33A9F431
:1025E000899CF0011124E45CFD4F008911890F5F83
:1025F0001F4F84819581A681B781E091BE05F0913E
:10260000BF0584839583A683B78301151105F9F06F
:10261000F8940F3FFFEF1F0731F422EE2093DD0502
:102620009092DE050EC0899CF0011124E45CFD4F00
:10263000168A892D806F8093DD051093DF05009346
:10264000DE0531E73093DC050E94430778948091E2
:102650002102811128C0F60180818E3421F58091FC
:10266000C005882301F1889EF0011124E45CFD4F30
:1026700096899860968BE0914001F091410102802B
:10268000F381E02D24E1829FE00DF11D1124E590FE
:10269000F4904CE050E067E571E0C70103960E94BA
:1026A0006F370E94162380912102833009F073C096
:1026B000F7018081833509F073C0E0914001F0910A
:1026C00041010188F289E02DB496A591B4918091E1
:1026D000B70580FD03C08C9182FF21C08091B705B2
:1026E0008E7F8093B705EB81FC8180818B7F808317
:1026F0008C918B7F8C9329E4E22E21E0F22E0AE864
:1027000012E520EE3FEF42E064E870E083E290E003
:102710000E94FC2B0E941623612C712C41C0E09179
:10272000BE05F091BF0580819181A281B381808730
:102730009187A287B3870E94C8328091B7058160D4
:102740008093B705EB81FC8180818460808399E36D
:10275000E92E91E0F92E0AE812E520EE3FEF42E083
:1027600064E870E083E290E00E94FC2B0E94162354
:102770008091B70581FD19C0FAEA26EE36E941E0FD
:10278000F150204030404040D9F7000084EB94E005
:102790009C838B830EC0E4EBF4E0FC83EB8309C0E5
:1027A00024EB34E03C832B8304C044EB54E05C8393
:1027B0004B8300E21EE40E94C82D8111FCCF5FEF25
:1027C00080E792E0515080409040E1F700C0000067
:1027D0001092090210920A0210920B0210920C023F
:1027E0008091B70580FF24C0F8948091B70581FFE0
:1027F00004C0C3010E94FB3203C0C3010E94103217
:102800003C01892B21F08091B70580FD10C088E63E
:1028100090E00E94131F8091B7058E7F8093B705CB
:10282000E981FA8180818B7F80830E9416237894CE
:1028300080913F0181FF5AC080912102813009F0CF
:1028400055C0F0902406FF2009F450C00032FEE489
:102850001F0709F049C023E12F1518F01092240634
:1028600002C083E1F82E40913B0150913C01415060
:102870005109A12CB12CC12CD12CE12C01E02AE171
:1028800030E06AE070E085E090E00E94572ACF2CAB
:10289000EB80FC8000E010E020EE3FEF42E06AE0D9
:1028A00070E085E090E00E94442C4B815C8184E0E4
:1028B000443B580769F0FA0101900020E9F7CF0185
:1028C00044978417950739F4E3EBF4E0FC83EB833A
:1028D00002E21EE402C000E010E02B813C812F5F89
:1028E0003F4F3C832B8302C00E5F1F4F31EA2316FC
:1028F00030EF330639E14306510430F00E94D01620
:10290000212C312C210105C04FEF241A340A440A2E
:10291000540A80913F0184FF04CE809121028111ED
:1029200000CE8091090290910A02A0910B02B09111
:102930000C02813854E895075EE1A507B10538F02F
:10294000809170008111EDCD0E94CB05EACD0196FA
:10295000A11DB11D8093090290930A02A0930B025E
:10296000B0930C02DECD1F920F920FB60F9211247E
:102970002F933F934F935F936F937F938F939F9387
:10298000AF93BF93EF93FF93359929C080910001D6
:10299000909101019093BF058093BE05109224068B
:1029A0001092DD050E94430760E08091B6050E9409
:1029B000BE048091BE059091BF0590930101809364
:1029C000000188EF95E09093BF058093BE051092BB
:1029D000090210920A0210920B0210920C02FF914F
:1029E000EF91BF91AF919F918F917F916F915F9187
:1029F0004F913F912F910F900FBE0F901F90189500
:102A00002A9A229A2D9A259A2498239A8DB58E7FF8
:102A10008DBD83E58CBD8DB508958EBD0DB407FECB
:102A2000FDCF8EB508958FEF0E940D150895FB011F
:102A3000E40FF51F39E06E177F0761F0229198E0EF
:102A4000880F482F422747FD8327220F9150C1F757
:102A50008F77F1CF08950E9400150895A5E0B0E0AA
:102A6000E4E3F5E10C94DB344A835B836C837D8380
:102A7000806489830E940D158D810E940D158C81C3
:102A80000E940D158B810E940D158A810E940D15E3
:102A900041E050E0BE016F5F7F4F80E00E9417155C
:102AA00044E050E0BE016E5F7F4F0E941715880F13
:102AB00081600E940D151FEF0E941315115011F037
:102AC00087FDFACF2596E3E00C94F734CF932A984C
:102AD0000E942E15C82F2A9A0E9413158C2FCF9171
:102AE0000895EF92FF920F931F93CF93DF938FEF91
:102AF0009FEFDC018093110690931206A0931306BA
:102B0000B093140610921506809110068E7F809364
:102B10001006CAE00E941315C150E1F7DAE040E068
:102B200050E0BA0180E00E946615813031F0D1504A
:102B3000B1F78093B402C1E091C084EBE82E82E04B
:102B4000F82E1AE02A984AEA51E060E070E088E046
:102B50000E942E15D82F8130C1F4870184E0E80E41
:102B6000F11C0E941315F80181938F01EE16FF06E8
:102B7000C1F78091B602813031F48091B70210E044
:102B80008A3A11F402C010E0D6E02A9A0E94131586
:102B90008D2F8B7F813061F08FEF810F112311F02A
:102BA000182FD0CFD63020F0F701D083C2E056C026
:102BB0000FEF13E040E050E0BA0187E30E94661592
:102BC000D82F8230A8F540E050E060E070E489E260
:102BD0000E946615811127C02A9840E050E0BA0192
:102BE0008AE30E942E15D82F0E9413158093B802F5
:102BF0000E9413158093B9020E9413158093BA02A4
:102C00000E9413158093BB022A9A0E94131580918B
:102C1000B80286FB882780F99091100680FB90F916
:102C20009093100605C00150110921F6C3E016C0AB
:102C3000D53041F440E050E0BA0181E00E946615D1
:102C400081110BC040E052E060E070E080E10E9442
:102C50006615882319F0C5E001C0C4E08C2FCDB7FC
:102C6000DEB7E6E00C94F434CF93DF93AB01BC0104
:102C70002A988091100680FD07C089E0440F551FF7
:102C8000661F771F8A95D1F781E10E942E15811169
:102C900015C00E9413158E3FE1F7C4EBD2E00E94ED
:102CA0001315899384E0C43BD807C9F70E94131514
:102CB0000E9413152A9A0E94131580E0DF91CF918C
:102CC0000895CF93DF93AB01BC012A988091100641
:102CD00080FD07C089E0440F551F661F771F8A9546
:102CE000D1F788E10E942E15811120C00E94131592
:102CF0008EEF0E940D15C4EBD2E089910E940D1554
:102D000084E0C43BD807C9F70E9413150E9413152D
:102D10000E941315982F9F71953041F40E9413154E
:102D20008823E1F32A9A0E94131580E0DF91CF9166
:102D300008950F931F93CF93C82F00E018EF21E061
:102D400043E050E065E070E08FE090E00E94AC2A44
:102D5000CC23F1F0C0E160911106709112068091D0
:102D60001306909114060E946116882319F0C15031
:102D700091F7FFCF1092150600E010E021E043E04C
:102D800050E065E070E08FE090E00E94AC2A03C064
:102D900081E08093150680E0CF911F910F910895F7
:102DA00080911506882321F081E00E949916FACFC0
:102DB0000895CF92DF92EF92FF92CF93C0901106C9
:102DC000D0901206E0901306F0901406C616D706AF
:102DD000E806F90611F48FEF18C06B017C010E9420
:102DE000D016C0E0C701B6010E943416C150882336
:102DF00019F0C111F7CFEFCFC0921106D092120691
:102E0000E0921306F092140680E0CF91FF90EF90CD
:102E1000DF90CF900895CF92DF92EF92FF92C09013
:102E20002F02D0903002E0903102F0903202611512
:102E300071058105910569F4809133029091340206
:102E4000A7019601281B390B41095109CA01B90193
:102E50000FC09B01AC012250310941095109A091D9
:102E60003702B0E00E94B9346C0D7D1D8E1D9F1D90
:102E7000FF90EF90DF90CF900895A0E0B0E0E3E402
:102E8000F7E10C94CE3460E070E0CB010E94D916DB
:102E90008111E8C0D091760480907A0490907B04F0
:102EA000A0907C04B0907D04C501B4010E94D916A5
:102EB000C82F8111D9C0E091C502F091C60284E00B
:102EC000F695E7958A95E1F7F0933402E0933302A3
:102ED0008091CA029091CB02009719F0A0E0B0E077
:102EE00008C08091D8029091D902A091DA02B091E5
:102EF000DB0280932B0290932C02A0932D02B093BF
:102F00002E02C090C202D090C302E12CF12CA091FD
:102F1000C40220912B0230912C0240912D0250913D
:102F20002E02B0E00E94B9342B013C01B501A4018E
:102F30004C0D5D1D6E1D7F1D8F0120E030E0D30123
:102F4000C201840F951FA61FB71F800F911FA21FDC
:102F5000B31F80932F0290933002A0933102B0935D
:102F600032028091C7029091C802009719F0A0E048
:102F7000B0E008C08091D4029091D502A091D60211
:102F8000B091D70284199509A609B7098C199D0932
:102F9000AE09BF09801B910BA20BB30B80932302D8
:102FA00090932402A0932502B09326028091C1023F
:102FB000809337028091BF029091C00290933602B5
:102FC0008093350240932702509328026093290290
:102FD00070932A028FEF9FEFDC0180931606909387
:102FE0001706A0931806B0931906DD3038F4DB30CD
:102FF00098F4D43029F0D630C9F502C0DE30B1F5EE
:10300000E091BE05F091BF051482158216821782E9
:10301000809110068D7F13C08091E0029091E102B3
:10302000A091E202B091E302E091BE05F091BF05EC
:1030300084839583A683B7838091100682608093F2
:103040001006E091BE05F091BF0584819581A681AF
:10305000B7818093380290933902A0933A02B093DB
:103060003B0205C0C1E003C0C2E001C0C3E08C2F39
:10307000CDB7DEB7E0E10C94EA348F929F92AF9225
:10308000BF92CF92DF92EF92FF922091100621FF24
:103090000EC042E0660F771F881F991F4A95D1F72F
:1030A000CC24CA94DC2CEC2C5FE0F52E09C0660F12
:1030B000771F881F991FCC24CA94DC2CE12CF12C9B
:1030C000209135023091360240E050E00E945434A5
:1030D0004B015C018091270290912802A091290266
:1030E000B0912A02BC01CD01620F731F841F951F8E
:1030F0000E94D916F401EC54FD4F80819181A28188
:10310000B381BC01CD016C217D218E219F21FF90D7
:10311000EF90DF90CF90BF90AF909F908F900895E9
:10312000AAE0B0E0E6E9F8E10C94CC341C016A8333
:10313000E091BE05F091BF05C480D580E680F780A0
:103140008091160690911706A0911806B091190665
:10315000C816D906EA06FB0651F0C0921606D092B0
:103160001706E0921806F092190610921A0680913E
:103170001A06882389F020911A0230911B023E839F
:103180002D832215330598F02215330529F481305B
:1031900019F43A81332359F0C701B6010E940B1785
:1031A0002B013C0110E01E821D82198240C000915B
:1031B00010028090160290901702A0901802B09012
:1031C0001902C0901102D0901202E0901302F09008
:1031D0001402109115021982240135018FEF481A4B
:1031E000580A680A780AC501B4010E94D91690E20B
:1031F000099FF0011124EC54FD4F4081442309F450
:10320000E9C0453EC9F4B0960F5F0031B1F7C11473
:10321000D104E104F10409F0CCC0812F90E02091A9
:103220003302309134028217930708F0BBC01F5F4E
:103230005301420100E0D0CF83858F3009F053C0A5
:10324000AA81AA2301F3842F90E001978F70992718
:10325000BDE0B89FB001B99F700D11246C547B4F35
:103260009F017A876987CF010A969C838B83F887B1
:10327000EF83AF81B88511965C91A985BA855D937E
:10328000BA87A9878F819885029698878F83AB81AB
:10329000BC818A179B0769F7CB0105969C838B83BA
:1032A000CF010C96D9011E965C91AB81BC815D93D8
:1032B000BC83AB832E5F3F4F8217930799F7848DB2
:1032C000DB011B968C931B97868D1C968C931C9709
:1032D00046FF02C01D961C924F70413009F093CFFB
:1032E00031E0398390CFB981BB2361F02D813E81DC
:1032F0002215330509F470C02F5F3F4F3E832D83A5
:10330000198281CF4E3229F49181903211F484FDDB
:103310007ACF83FD78CF8D819E8182159305D9F573
:10332000CF0164EB74E0AB01DC012D91CD01DA013A
:103330002D93AD01B4E04F3B5B07B1F71092BF0492
:103340002A81222309F44AC01092C0048091BE044D
:103350008093BF048091BD048093BE048091BC041F
:103360008093BD048091B4048E3219F08EE2809374
:10337000BC0424EB34E0DB018D91BD01803221F0EF
:10338000D9018C932F5F3F4FDB018C918111F3CFDB
:10339000D9011C9223C02D813E812F5F3F4F3E8378
:1033A0002D8331CF90911006892F827091FD3FCFF0
:1033B0006EC080913702181708F439CFC701B601E3
:1033C0000E943D186B017C010E940B172B013C01F0
:1033D00010E02DCF80E005C082E003C03E822D8248
:1033E00081E0A091BE05B091BF054489558960E098
:1033F00070E0BA0155274427228D338D2901612CB5
:10340000712C44295529662977294D935D936D9335
:103410007C93139751963C922E925097448D558DE4
:10342000668D778D52964D935D936D937C935597F2
:1034300093859093B805268937893093BC052093EE
:10344000BB05208D318D3093BA052093B9058823B3
:10345000E9F0AD81BE81B0931B02A0931A020093E4
:1034600010028092160290921702A0921802B09257
:103470001902C0921102D0921202E0921302F0924D
:1034800014021093150280931A0601C080E02A9658
:10349000E2E10C94E834A0E0B0E0E1E5FAE10C945C
:1034A000D6346B017C01E091BE05F091BF058485A7
:1034B0009585A685B785C816D906EA06FB0660F489
:1034C00080819181A281B38180879187A287B38710
:1034D0001486158616861786C091BE05D091BF0545
:1034E0000C851D852E853F85688579858A859B8518
:1034F000C016D106E206F306B1F00E943D186887B7
:1035000079878A879B87E091BE05F091BF05848506
:103510009585A685B7850196A11DB11D84879587E0
:10352000A687B787D9CFCDB7DEB7E8E00C94F234E1
:10353000A9E0B0E0EEE9FAE10C94CC34E091BE05EC
:10354000F091BF05428853886488758844155505F5
:103550006605770518F080E090E0E2C019016A0185
:103560007B018D8320913702A0913502B091360204
:10357000AD0160E070E04E835F836887798730E05B
:103580000E94A3344B015C01C301B2016C197D0997
:103590008E099F0969837A838B839C83C701B60157
:1035A000A50194010E94543429013A01A501940116
:1035B000C301B2010E941034C61AD70AE80AF90AF8
:1035C000C701B6012E813F81488559850E94543438
:1035D00049015A012E813F8148855985C501B401B1
:1035E0000E941034C61AD70AE80AF90AC301B201C8
:1035F0000E944B1AE091BE05F091BF056085718570
:10360000828593850E940B17680D791D8A1D9B1D6D
:103610000E94D91604EB14E01F821E828E819F81C6
:103620008215930509F44BC08091350290913602C2
:10363000A0E0B0E0C816D906EA06FB06C0F17D811D
:103640007130E1F08FEF881A980AA80AB80A8091C1
:10365000370290E0A0E0B0E088169906AA06BB0603
:1036600098F09FEF491A590A690A790AC301B20111
:103670000E944B1A812C912C540106C080E00E94BC
:1036800099168823F9F267CFE091BE05F091BF0546
:1036900060857185828593850E940B17680D791D61
:1036A0008A1D9B1D0E94D916C12CD12C76014981FF
:1036B0005A816B817C81452B462B472B21F45D8100
:1036C000513061F526C0F601EC54FD4F6D8161303B
:1036D00019F4D8018C9102C08081F801808349815E
:1036E0005A816B817C81415051096109710949837B
:1036F0005A836B837C836E817F816F5F7F4F7F8373
:103700006E837FEFC71AD70AE70AF70A0F5F1F4FCA
:1037100085CF80E00E94991681111DCF8E819F81F7
:103720002996E2E10C94E834AAE1B0E0EAE9FBE191
:103730000C94CC349C878B87788F6F8BDC018D90B9
:103740009D90AD90BC90BFEF8B1A9B0AAB0ABB0A51
:1037500080911006209035023090360281FF11C012
:1037600036942794369427942FEF3FEF4FEF5FE086
:103770002F83388749875A8744E050E05E834D8322
:103780000EC0369427948FEF9FEFA0E0B0E08F83B8
:103790009887A987BA87A2E0B0E0BE83AD836101B4
:1037A000E12CF12CC501B401A70196010E9454340B
:1037B00029013A01A7019601C301B2010E94103408
:1037C00069837A838B839C8380912702909128025E
:1037D000A0912902B0912A02480E591E6A1E7B1E32
:1037E00040912702509128026091290270912A028B
:1037F00080912B0290912C02A0912D02B0912E026B
:10380000840F951FA61FB71F481659066A067B0628
:1038100008F0C4C0C301B2010E94D916C501B401A9
:10382000A70196010E9454347A8F698F80902702F5
:1038300090902802A0902902B0902A0200912B02B9
:1038400010912C0220912D0230912E02800E911E9B
:10385000A21EB31EA501940121503109410951094D
:103860002D873E874F87588B209123023091240269
:103870004091250250912602298B3A8B4B8B5C8B11
:1038800080903702912CA12CB12CAD81BE81A69FD6
:10389000A001A79F500DB69F500D11245E8B4D8B3C
:1038A00000E010E0498D5A8D4215530508F061C0C3
:1038B0002D853E854F855889421653066406750648
:1038C000E9F469897A898B899C89A50194010E9410
:1038D0005434CA01B901A70196010E945434DC0195
:1038E000CB010196A11DB11DE98DFA8DAF0160E0FC
:1038F00070E084179507A607B707D8F1ED89FE8910
:10390000E00FF11FEC54FD4F80819181A281B381C2
:103910002F81388549855A8582239323A423B52393
:103920004D815E81040F151F892B8A2B8B2BD1F4BF
:10393000C980DA80EB80FC80898D9A8DC80ED91EF3
:10394000E11CF11CAB85BC85CD92DD92ED92FC9221
:103950001397EF89F88D408251826282738280E0F2
:1039600090E01EC0298D3A8D2F5F3F4F3A8F298FEF
:1039700099CF89819A81AB81BC818C0D9D1DAE1D33
:10398000BF1D89839A83AB83BC839FEF491A590A71
:10399000690A790A812C912C540122CF81E090E0B0
:1039A0006A96E2E10C94E834A9E1B0E0EAEDFCE1CA
:1039B0000C94CC345C016A017B0120911602309199
:1039C000170240911802509119022E873F87488BA9
:1039D000598B0091100210E00F5F1F4F0F701127DD
:1039E0000115110541F42F5F3F4F4F4F5F4F2E8759
:1039F0003F87488B598B8091100681FD0DC08FEF5A
:103A00009FEFA0E0B0E08A8B9B8BAC8BBD8BA2E0DC
:103A1000B0E0BD87AC870CC02FEF3FEF4FEF5FE00A
:103A20002A8B3B8B4C8B5D8B44E050E05D874C8751
:103A300019821A821B821C82BE016B5F7F4FCE01EE
:103A400001960E94941B892B29F060E070E080E0D1
:103A500090E046C16E857F85888999890E94D91634
:103A600085E0000F111F8A95E1F7C8018C549D4F26
:103A70009A87898789819A81AB81BC81E985FA859A
:103A8000B58BA48B938F828F48E050E0B501CF01B6
:103A90000E947E3743E050E06AE272E089859A85B1
:103AA00008960E946F37A985BA855C96CD92DD9203
:103AB000ED92FC925F9780E21B968C9380E00E94CF
:103AC00099168111C2CF89809A80AB80BC80C501D4
:103AD000B4010E940B176E8B7F8B888F998F20907B
:103AE000350230903602B0913702BB87910140E039
:103AF00050E0C701B6010E945434EB854E2E512C84
:103B0000612C712CCA01B901A30192010E945434A5
:103B10008901FB85F29D9001F39D300D112440E059
:103B200050E0C701B6010E945434672B682B692B03
:103B300011F401501109C1016C857D850E942C345E
:103B40009B0140E050E0C501B4010E9454348091D3
:103B5000270290912802A0912902B0912A02820F97
:103B6000931FA41FB51F8D839E83AF83B887612CDD
:103B7000712C1B862C853D851901412C512C80917F
:103B80003502909136026C857D850E942C349B0114
:103B900040E050E069817A818B819C810E9454349D
:103BA0009B01AC01C201B1010E9410346B017C0188
:103BB0008D809E80AF80B884BE016B5F7F4FCE0149
:103BC00001960E94941B892B21F03B853F5F3B8728
:103BD00083018D819E81AF81B88588169906AA06DA
:103BE000BB0621F0C501B4010E94D91680911006D0
:103BF000F601EC54FD4F60167106A0F481FF0DC074
:103C000089819A81AB81BC812A893B894C895D89F4
:103C100082239323A423B5230BC089819A819183A6
:103C200080830FC081FF09C08A899B89AC89BD89C7
:103C300080839183A283B38304C0AFEFBFEFB183CE
:103C4000A08380E00E94991680912B0290912C0213
:103C5000A0912D02B0912E02BC01CD01680D791DFD
:103C60008A1D9B1D0E946116BFEF6B1A7B0A061509
:103C7000170508F084CFEB85EE2331F16E857F8543
:103C8000888999890E94D91620913702809135023E
:103C900090913602289FA001299F500D1124C80140
:103CA0000196489F9001499F300D589F300D112477
:103CB000C901A0E0B0E0E985FA85848F958FA68FD1
:103CC000B78F81E00E94991680911A0290911B0291
:103CD00060E001960E9490186E897F89888D998D89
:103CE0006996E2E10C94E834ABE0B0E0EAE7FEE18B
:103CF0000C94CE341B861A866115710581059105D9
:103D000021F460E070E0CB017BC04091370220914C
:103D1000350230913602429FF001439FF00D11248D
:103D20008F0120E030E098011127002706171707C0
:103D30002807390730F32B013C01E091BE05F091D3
:103D4000BF058091160690911706A0911806B091B4
:103D5000190684839583A683B78380E090E000E012
:103D600010E04E012AE0820E911C22E2C22E22E0D7
:103D7000D22E34EBA32E34E0B32E7C012FEFE21AC7
:103D8000F20A60E00E9490188823B1F09F928F920F
:103D9000DF92CF92BF92AF920E94AF378A859B8508
:103DA0000F900F900F900F900F900F90081719071A
:103DB00008F48C01C701E1CF81E0E816F10409F4B1
:103DC000A0CF0F5F1F4F003127E2120708F099CFF5
:103DD0001F930F9389E192E09F938F938E010F5F62
:103DE0001F4F1F930F930E948D37B301A201C8018B
:103DF0000E94D41C0F900F900F900F900F900F9077
:103E00002B96E0E10C94EA34FC01680F791F80E006
:103E1000E617F70739F09191980F981708F49F5F0C
:103E2000892FF6CF08952091C00025FFFCCF9093F5
:103E3000C5008093C40082E28093C00088E1809333
:103E4000C10087E08093C2008091C00087FF03C05B
:103E50008091C600F9CF08959091C00095FFFCCFE6
:103E60008093C60008950F931F93CF93DF93EC01C7
:103E70008C01060F171FC017D10721F089910E94EE
:103E80002C1FF9CFDF91CF911F910F910895CF9201
:103E9000DF92EF92FF92CF93DF939B01FC0152EFF1
:103EA000C52E59E4D52E52E0E52EF12C50E0A6B1F6
:103EB000A072B0E0A417B50711F5A1E0CA1AD108A5
:103EC000E108F108F1F0A091C000A7FFF0CFA091A8
:103ED000C000D091C600A4FD16C0CA2FC870A3FDB3
:103EE00014C02115310531F40E94041FD81771F058
:103EF000C0E80CC0D083215031093196D8CFC1E041
:103F000005C0C2E003C0C3E001C0C4E08C2FDF9154
:103F1000CF91FF90EF90DF90CF900895A1E0B0E0B7
:103F2000E4E9FFE10C94DC3440E20E94471F8983FE
:103F30008FE99FE00197F1F700C000008981882395
:103F400091F08EE40E942C1F80910F028823B9F01B
:103F50008EE40E949E058981805D8983CE01019651
:103F60000E947A260CC081E40E942C1F80910F02CF
:103F7000882331F081E40E949E0580E001C08FEF2C
:103F80002196E2E00C94F8340F931F93CF93DF93C4
:103F9000EC018B0180910F02882351F0442321F022
:103FA00085E40E949E050CC083E40E949E050AC021
:103FB0008FE79CE00197F1F700C00000442311F067
:103FC00085E401C083E40E942C1F8FE193E00197F8
:103FD000F1F700C00000B801CE010E94331FB80104
:103FE000CE010E94041F0E942C1FDF91CF911F91D0
:103FF0000F9108954096FC01A591B4918C91846035
:104000008C9380E090E0089581E08093210280937A
:1040100020027894E0914001F09141010580F68101
:10402000E02D099580E090E0089580912102813093
:1040300051F480911E0290911F020A9790931F02E3
:1040400080931E0204C010920F0210922002109260
:104050002102E0914001F09141010190F081E02DB9
:10406000099580E090E008951092210280911E024F
:1040700090911F020A9790931F0280931E028091D5
:104080002002882339F083E08093210210925001AE
:1040900010924F0180912102E0914001F091410185
:1040A00095E0899FE00DF11D11240190F081E02D34
:1040B000099580914F0190915001089582E080937D
:1040C0002102E0914001F09141010284F385E02D4D
:1040D000099580E090E0089580E090E00895FC016B
:1040E00080911B0690911C06893C910568F081E047
:1040F000809321027894E0914001F0914101058084
:10410000F681E02D099508C0889748F07096A59132
:10411000B4918C9184608C9380E090E008958FEF4F
:104120009FEF0895FC018285838781858287808542
:1041300081878EE2808714860895EF92FF920F9315
:104140001F93CF93DF9380911C0290911D02892BC6
:1041500009F45AC060E080911E0290911F020E94F3
:104160009018882309F4C6C060E270E08FE090E008
:104170000E94682C20911C0230911D0282E491E083
:104180009F938F93C9010197EAE0F0E0BF010E947D
:104190002C346F5F7F4F7F936F9380911E029091BD
:1041A0001F02BF010E942C346F5F7F4F7F936F937C
:1041B0003F932F9381E792E09F938F9384EB94E05A
:1041C0009F938F930E948D3724EB34E040E050E0C2
:1041D0006FEF7FEF81E00E94992C6DE270E08FE03D
:1041E00090E00E94682CC0911E02D0911F028DB7F2
:1041F0009EB70C960FB6F8949EBF0FBE8DBF8FE092
:10420000E82E85E0F82E44C060E080911C02909179
:104210001D020E949018882309F49CCF80911C02F3
:1042200090911D02019690931D0280931C02ECCF89
:1042300060E0CE010E949018882309F44DC080915F
:10424000B8052091BC0484FD3AC08EEE94E0FC01D8
:104250003491231731F10396E816F906C1F70DE7FB
:104260001FEE203291F184EB94E00E949220809125
:104270004F019091500124EB34E04AE852E5C81711
:10428000D90741F560EF7FEF82E00E94992C2196DB
:1042900080911E0290911F020A96C817D90740F21A
:1042A00025C03196E4913091BD043E13D4CFFC017A
:1042B0003296E4913091BE043E13CDCF03C00FEF90
:1042C00017E0CFCF00EE17E0CCCF2093BF041092C1
:1042D000C004CDCFB801D8CF24E632E04AE852E599
:1042E00060EE77E082E00E94712CD1CFD0931F0264
:1042F000C0931E0280E090E0CDB7DEB7E6E00C94FC
:10430000F43480911E0290911F028431910538F09F
:10431000449790931F0280931E020E949D2080E08C
:1043200090E0089510921F0210921E020E949D209C
:1043300080E090E0089580911C0290911D02019709
:104340006AE070E00E942C342AE0269FC001279F7B
:10435000900D112490931F0280931E020E949D20B5
:1043600080E090E00895A5E0B0E0E9EBF1E20C9484
:10437000CC3480E090E00E948629198204E110E0AC
:1043800024E130E03D832C838C809D803AE0830ED5
:10439000911CAC80BD808AE0A81AB1082FEF3FEFD6
:1043A000A801B401C5010E944B2A68019AE0C90E18
:1043B000D11C78012AE0E21AF1082FEF3FEFA601A5
:1043C000B7018C819D810E94412A0E94C82D8111D4
:1043D000FCCF0E94C82D8823E1F30E94342F609304
:1043E0001B0670931C0680931D0690931E0620EEFC
:1043F00037E0A801B401C5010E944B2A20EE37E046
:10440000A601B7018C819D810E94412A60911B0603
:1044100070911C0680911D0690911E0639813230E4
:10442000D1F0333019F1313051F03B011C01809152
:104430003B0190913C0144979D838C8324C02B01C8
:10444000280E391E3694279400913D0110913E01AB
:104450000451110918C0460E571E569447949B8369
:104460008A8324E130E03D832C830DC0660E771EE5
:10447000769467942A813B81820F931F9C01369525
:1044800027953B832A833FEF89E698E131508040AE
:104490009040E1F700C0000029812F5F298324307C
:1044A00009F072CF0E94C82D8111FCCF60913B01B1
:1044B00070913C0180E090E00E9418366B017C0115
:1044C000C201861997099D838C83BC01990F880BC3
:1044D000990B0E941A364B015C0120E030E040E26B
:1044E00052E4C701B6010E9403359B01AC01C5012E
:1044F000B4010E947035A70196010E94A6360E9461
:10450000E2352C813D81621B730B77FF02C06F5F28
:104510007F4F75956795661A770A460E571E60910C
:104520003D0170913E0180E090E00E9418366B01E1
:104530007C018A819B81821993099D838C83BC01B4
:10454000990F880B990B0E941A364B015C0120E0F1
:1045500030E040E252E4C701B6010E9403359B01FE
:10456000AC01C501B4010E947035A70196010E94FB
:10457000A6360E94E2352C813D81621B730B77FFCA
:1045800002C06F5F7F4F75956795261A370A8A813B
:104590009B81860F971F9B838A839F938F933F9264
:1045A0002F925F924F927F926F9285E492E09F9359
:1045B0008F9384EB94E09F938F930E948D3760914B
:1045C0003D0170913E017695679524EBE22E24E043
:1045D000F22E00E010E02FEF3FEF41E084E190E0A9
:1045E0000E94212C0FB6F894DEBF0FBECDBF0E94F3
:1045F000C82D8823E1F3B3018DEB91E00E94A63D25
:10460000B20189EB91E00E94A63DB1018BEB91E0F4
:104610000E94A63D6A817B8187EB91E00E94A63DC6
:1046200080E090E02596E2E10C94E834A7E1B0E068
:10463000ECE1F3E20C94CC341D8A80912102E091EC
:104640004001F091410195E0899FE00DF11D112499
:1046500084819D89981708F082C0228133819D89C9
:1046600084E1989FA0011124DE01119680E090E082
:10467000FA01E80FF91FE20FF31FE491ED930196A1
:1046800084319105A9F7E989FA89E080E1FE63C0E8
:10469000E2FE08C0EFE1F0E0FC87EB8780EE9FEFE1
:1046A000988B8F874B845C848D809E80E985FA850A
:1046B000FF8BEE8B6B807C802F803884260C371C20
:1046C000AD84BE84E0FAEE24E0F89F01280D391D88
:1046D000620101E0A101B401C3010E94572AC9800F
:1046E000DA802F853889C40106976E897F8976958F
:1046F0006795680F791F7601820142E0C3010A962F
:104700000E94212CF6018081843429F58181803337
:1047100011F12401F8E14F0E511C310182E0681AB9
:10472000710898E0890E911CE2E12E1A310805E12A
:1047300015E09201A301B401C1010E94C12CF60150
:1047400083818C3341F400E018EF9201A301B4019E
:10475000C1010E94F029FD89FF5FFD8B6ECF679636
:10476000E2E10C94E8344096FC01A591B4918C915F
:1047700082FB992790F9909590FB82F98C93809118
:10478000B70582FB992790F9909590FB82F9809369
:10479000B7050E94162380E090E008954096FC0142
:1047A000A591B4918C9182FF08C08091B70581607A
:1047B0008093B7058C918B7F09C08091B70580FFEE
:1047C00008C08E7F8093B7058C9184608C930E9483
:1047D000162380E090E008954096FC01A591B491E5
:1047E0008C9182FB992790F9909590FB82F98C939C
:1047F0000E94162380E090E00895AF92BF92CF927E
:10480000DF92EF920F93CF93DF93CBE3D1E0488118
:1048100059814B505109A12CB12C8AE8C82E82E550
:10482000D82EE12C01E028E131E068E270E08AE076
:1048300090E00E94572A488159814B50510999E5CF
:10484000C92E9EECD92E00E028E131E068E270E04C
:104850008AE090E00E94572A488159814C505109C2
:1048600027E131E069E270E08BE090E00E94572A96
:104870000E9416238FEF9FEF9093500180934F017A
:104880000E949D20DF91CF910F91EF90DF90CF900C
:10489000BF90AF900895AF92BF92CF92DF92EF9208
:1048A0000F93CF9340913B0150913C014B505109E4
:1048B000A12CB12C8AE8C82E82E5D82EE12C01E08B
:1048C00028E131E068E270E08AE090E00E94572A37
:1048D00040913B0150913C014B50510999E5C92E43
:1048E0009EECD92E00E028E131E068E270E08AE039
:1048F00090E00E94572A40913B0150913C014C505E
:10490000510927E131E069E270E08BE090E00E941C
:10491000572A609140017091410140E050E020E051
:1049200030E080912102FB0195E0899FE00DF11DAF
:104930001124848190E002972817390750F50280EE
:10494000F381E02DE40FF51F7096A591B491E091ED
:104950003F01F0E0022E02C0F595E7950A94E2F7D8
:104960008C91E0FB82F98C9390912102FB01C5E0D0
:104970009C9FE00DF11D1124E481F0E033972E1788
:104980003F0711F48B7F8C932F5F3F4F4C5E5F4F3F
:10499000C8CF0E941623CF910F91EF90DF90CF9058
:1049A000BF90AF900895A0E0B0E0E9EDF4E20C9480
:1049B000D434CBE3D1E04881598146505109A12C30
:1049C000B12C8AE8C82E82E5D82EE12C01E025EF33
:1049D00030E064E670E085E090E00E94572A48816C
:1049E00059814650510999E5C92E9EECD92E00E017
:1049F00025EF30E064E670E085E090E00E94572A01
:104A0000488159814750510924EF30E065E670E054
:104A100086E090E00E94572A2CE3E22E22E0F22E5C
:104A20000AE812E528E03CEF42E069E670E086E43F
:104A300090E00E94FC2B688179816850710928E020
:104A40003CEF4AE750E087E090E00E944B2A0E944A
:104A50001623CDB7DEB7EAE00C94F034A0E0B0E066
:104A6000E4E3F5E20C94D434EC01162F60911F06B8
:104A70007091200680913D0190913E0140978617EC
:104A8000970718F481E0809323069B01295F3F4F2D
:104A900040913B0150913C014B505109A12CB12C4C
:104AA0008BE7C82E85E2D82EE12C01E0809121060B
:104AB000909122060E94572A60911F06709120064D
:104AC00080912106909122067E01112341F00BE78F
:104AD00015E22FEF3FEF41E00E94FC2B07C00BE7F0
:104AE00015E22FEF3FEF41E00E94212C80911F063D
:104AF0009091200608969093200680931F0620919F
:104B000023062223E1F020913D0130913E012850FF
:104B100031092817390768F480912102843019F48B
:104B20008AE090E002C08CE191E0909320068093AF
:104B30001F0680911F06909120060E947A29CDB70A
:104B4000DEB7EAE00C94F03461E00E942E2508956F
:104B5000A0E0B0E0EEEAF5E20C94D43484E190E019
:104B600090932206809321068CE191E09093200699
:104B700080931F060E94CF2844E050E060E270E07E
:104B800080911F06909120060E94602980911F0647
:104B9000909120060E947A290E94CB2880E090E024
:104BA0000E9486298EE0E82E82E0F82E00E010E0D8
:104BB00028E03CEF42E06AE070E084E190E00E948F
:104BC000FC2B92E0E92E92E0F92E28E03CEF41E048
:104BD00062E170E080EA90E00E94FC2BCBE3D1E040
:104BE0006881798128E03CEF4EE150E080E090E080
:104BF0000E944B2A0E9416232A813B8121503109B1
:104C0000488159814B505109A12CB12C6BE7C62E1C
:104C100065E2D62EE12C01E068E171E08AE090E0E7
:104C20000E94572A1092230660911F067091200659
:104C300080912106909122060E94682C8FE095E0D9
:104C40000E94A42570E8E72E0BE715E22FEF3FEF57
:104C500041E064E271E084E190E00E947D2BCDB7F9
:104C6000DEB7EAE00C94F034EF920F931F938BE7DA
:104C700095E20E9486298AE090E090932206809334
:104C800021069093200680931F0646E050E060E3E3
:104C900071E00E94602980911F06909120060E9479
:104CA0007A291092230660911F0670912006809148
:104CB0002106909122060E94682C8FE095E00E94C8
:104CC000A42580E8E82E0BE715E22FEF3FEF41E047
:104CD00062E170E08AE090E00E947D2B81E08093A9
:104CE0000F0284E08093210280E090E01F910F91F9
:104CF000EF90089560E00E942E250895A2E2B0E0B2
:104D0000E4E8F6E20C94D9348C01F62E82E28F1599
:104D100088F442E250E0B801CE0101960E947E374D
:104D200060E0CE0101960E942E258EEDF80E0E5DFC
:104D30001F4FECCF60E0C8010E942E25A296E5E04F
:104D40000C94F534A0E0B0E0E8EAF6E20C94D63436
:104D500080911D0690911E068D9768E170E00E947B
:104D60002C34C0911E02D0911F022A97C60FD71F64
:104D700061E0CE010E9490188091B80584FF67C061
:104D8000E091BE05F091BF05C080D180E280F38044
:104D9000C482D582E682F7828091B4048E3209F013
:104DA0003FC08091B5048E32D9F5C114D104E1041D
:104DB000F10439F48FE290E0909343018093420133
:104DC00037C060E080E090E00E949018E091BE055E
:104DD000F091BF0580819181A281B3818483958305
:104DE000A683B78300E010E061E0C8010E9490183C
:104DF000E091BE05F091BF0580819181A281B381D0
:104E0000C816D906EA06FB0629F4C482D582E682D2
:104E1000F78206C00F5F1F4F0F3F110529F7F5CF2F
:104E20004CE050E064EB74E082E491E00E947E3755
:104E300010921F0210921E0210921D0210921C026C
:104E40008FEF9FEF9093500180934F011CC0E4EBD4
:104E5000F4E001900020E9F73197BF01645B7440F2
:104E60006093240684EB94E00E947E26D093500148
:104E7000C0934F0180911E0290911F020A97909358
:104E80001F0280931E020E949D2061E0CE010E94BD
:104E9000901880E090E0CDB7DEB7E8E00C94F234F3
:104EA000EF92FF920F931F93CF930E944B2DC82F29
:104EB0000E9404298EEA91E00E94743D80933F0194
:104EC00081700E942C290E9424299F938F938EE247
:104ED00092E09F938F9384EB94E09F938F930E9433
:104EE0008D3784EBE82E84E0F82E00E010E02FEF01
:104EF0003FEF42E062E271E084E190E00E94212C09
:104F00000F900F900F900F900F900F90CC2379F08F
:104F10008DEB91E00E94823D019629F40E94CB28FE
:104F20000E94B32104C00E94C82D8111F7CFCF91F8
:104F30001F910F91FF90EF900895FF920F931F9391
:104F4000CF93DF93F0903F01F0FAFF24F0F8109236
:104F50003F0180912102A0914001B091410175E093
:104F6000879FA00DB11D112460E0262F30E014961C
:104F70008C91149790E0FC0132972E173F0714F59F
:104F80001296ED91FC91139774E1679FE00DF11D6E
:104F90001124709605911491E80103972817390799
:104FA0007CF4888182FB442740F950E0CA0101C0AB
:104FB000880F2A95EAF790913F01892B80933F0152
:104FC0006F5FD3CF60913F018EEA91E00E94883DF0
:104FD000888182FD0EC080913F018170F81661F1D9
:104FE0006FEF7FEF8DEB91E00E94A63D0E9450276E
:104FF00023C0CCE3D2E006E911E08EA580FF0EC00D
:105000004C8D5D8D6E8D7F8DC8010E949A3D68A587
:1050100079A5C80104960E94A63D06C04FEF5FEF38
:10502000BA01C8010E949A3D68960A5F1F4F82E04C
:10503000CC39D80711F7CFCF0E94152080E090E03F
:10504000CDB7DEB7E5E00C94F534A0E0B0E0EBE2DC
:10505000F8E20C94D4340E94BA2E362F272F609396
:105060001B0670931C0680931D0690931E0680916C
:105070002102A0914001B091410195E0899FA00DCE
:10508000B11D11241496AC901497832F922F009188
:105090001D0610911E0640E050E0B12CBA1451F1EB
:1050A00012962D913C911397240F351FF9013296DA
:1050B000C590D490F9013496E590F490F9013696B4
:1050C000C591D491F901389665917491C816D906A5
:1050D00068F4CC0DDD1D8C179D0740F4E016F10639
:1050E00028F46E0D7F1D0617170738F0B3944C5E39
:1050F0005F4FD4CF80E090E001C0C901CDB7DEB7EB
:10510000EAE00C94F03484B1836084B98AB18C6F86
:105110008AB987B18F6187B988B18B6088B98FE30D
:105120009CE90197F1F700C00000089544988FE5CD
:105130009AEE0197F1F700C00000449A8FE59AEECD
:105140000197F1F700C0000008959BB19370282FDC
:105150002C7F922B9BB995B19C7F8370892B85B94D
:105160004198419A089540982FEF89EF90E021509F
:1051700080409040E1F700C0000029B193B1409A0F
:105180002C7F892F8370822B0895429843980E9428
:10519000A528439A089589E20E94C528089588E2C7
:1051A0000E94C5280895CF93C82F429A4398892F0B
:1051B0000E94A5288C2F0E94A528439ACF9108957C
:1051C000CF9384B18C7F84B98AB183708AB9429AB3
:1051D00043980E94B328C82F0E94B328439A94B1E1
:1051E000936094B99AB19C6F9AB92C2F30E0322F0A
:1051F0002227A901482BCA01CF910895429A4398CA
:105200000E94A528439A08950E9483280E94962808
:105210002FEF8DEE92E0215080409040E1F700C0EA
:1052200000008AE30E94C52885E50E94FE2881E1EE
:105230000E94C5282FEF81EE94E0215080409040DD
:10524000E1F700C00000089583ED0E94C5280E9488
:10525000E0280E94E0280895CF93C82F86E30E949B
:10526000C528CC2321F0C13029F488E901C088E4A5
:105270000E94FE28CF910895A0E0B0E0E2E4F9E2B8
:105280000C94D6346C018B017A01E9018AE20E9408
:10529000C528C6010E94D328C7010E94D3288BE2EB
:1052A0000E94C528C8010E94D328CE010E94D3289D
:1052B0008CE20E94C528CDB7DEB7E8E00C94F2344A
:1052C000EF92FF920F931F93CF93DF937C018B019B
:1052D000EA0183E30E94C528C7010E94D328C801C0
:1052E0000E94D328CE010E94D328CDB7DEB7E6E0D6
:1052F0000C94F434CF93DF93EC0187E30E94C5282C
:10530000CE010E94D328DF91CF910895CF92DF92F2
:10531000EF92FF92CF93DF93EC01209151013091F6
:105320005201215031094091530150915401415093
:10533000510960E070E080E090E00E943C29C12CBF
:105340008CE2D82EEE24E394F12CCE010E94D328D7
:1053500081E0C81AD108E108F108B9F7DF91CF91CF
:10536000FF90EF90DF90CF900895CF92DF92EF9271
:10537000FF920F931F93DA01A81BB90B1196F90145
:10538000E61BF70B3196AE9F6001AF9FD00CBE9F1E
:10539000D00C1124E12CF12C0E943C29C114D10421
:1053A000E104F10449F0C8010E94D32881E0C81A41
:1053B000D108E108F108F2CF1F910F91FF90EF9013
:1053C000DF90CF900895CF93DF93EA019B01AC016A
:1053D0000E943C29CE010E94D328DF91CF910895ED
:1053E000A0E0B0E0E6EFF9E20C94CE347C01EB01F2
:1053F0003A0129016A01C81AD90A5901A61AB70A3D
:10540000CC0CDD1CAA0CBB1CA8010E94E329AC1427
:10541000BD04C8F4C601969587954501881A990A76
:10542000E614F70449F197FC03C021968C189D08F7
:105430008FEFE81AF80A8A0C9B1CA801BE01C7016D
:105440000E94E329EDCFC501969587954601881AFC
:10545000990AC415D50581F097FC05C08FEFE81AAD
:10546000F80A8A189B0821968C0C9D1CA801BE0185
:10547000C7010E94E329EDCFCDB7DEB7E0E10C9480
:10548000EA340F931F9389019A01AC010E94B52958
:105490001F910F9108950F931F93FB01BA0189018A
:1054A0009A01AF010E94B5291F910F9108954F9263
:1054B0005F926F927F928F929F92AF92BF92CF92A4
:1054C000DF92EF920F931F93CF93DF933C014B0139
:1054D000EA012901013021F486010E94B52916C094
:1054E0009601A2010E94412A9601A201B401CE01B7
:1054F0000E94412A9601A401BE01C3010E944B2AC9
:105500009601A201BE01C3010E944B2AEE20A1F028
:10551000A501B401C3010E94E329A501B201C301A1
:105520000E94E329A501B401CE010E94E329A5014F
:10553000B201CE010E94E329DF91CF911F910F911B
:10554000EF90DF90CF90BF90AF909F908F907F9023
:105550006F905F904F900895ADE0B0E0E2EBFAE21B
:105560000C94CC347C013B015D874C872B8781E018
:1055700090E09C01241B350B3A83298317014B01D2
:105580007C836B83270143E050E058874F839E83E1
:105590008D832D813E81215031093A872987CC8422
:1055A000DD84C60CD71C3B85313039F59801A60146
:1055B000B101C2010E944B2A9801A3018C859D85EF
:1055C000481B590BB101C2010E944B2A98014B8123
:1055D0005C81AC84BD84AE0CBF1CB50167018C85B9
:1055E0009D85C81AD90AC6010E944B2A9801A401B8
:1055F000B501C6010E944B2A38C0A801B601C101FD
:105600000E94E329A8016B817C81AC84BD84AE0C2F
:10561000BF1CC5010E94E329A801B601C2010E9476
:10562000E329A8016B817C8167012C853D85C21A25
:10563000D30AC6010E94E329A801B401C5010E9452
:10564000E329A80153018C859D85A81AB90AB501E3
:10565000C1010E94E329A801B501C2010E94E3290A
:10566000A801B401C6010E94E32929813A8137FFCC
:105670000BC02D813E8149815A818F819885480FC9
:10568000591F5A83498316C02D813E8189859A8589
:105690004C855D85841B950B880F991F0596498164
:1056A0005A81480F591F5A8349838C859D850197DC
:1056B0009D878C874D815E814F5F5F4F5E834D83F9
:1056C0008F819885029698878F8391E0491A5108B7
:1056D0004FEF241A340A8B819C8101969C838B8323
:1056E00091E0891A91084C855D85421753070CF0AB
:1056F00050CF2D96E2E10C94E8342F923F924F92D6
:105700005F927F928F929F92AF92BF92CF92DF92E1
:10571000EF92FF920F931F93CF93DF93FC01542ED0
:105720004901411102C055245394852D90E09C01FC
:105730008E179F0708F4CF0143E0220F331F4A95CD
:10574000E1F7AB0141505109240F351FAC01415025
:105750005109E5E05E9E400D511D11240E943C2937
:1057600085E0E89E70011124C12CD12CE0EAEE1AEC
:10577000F10822242394312C0C2C02C0220C331C5F
:105780000A94E2F7712CA12CB12CF701EA0DFB1D54
:10579000EA5EF84FC491D0E0C221D321412C20977A
:1057A00011F0C40101C0C8010E94D32843945410D1
:1057B000F6CF8FEFA81AB80AE5E0AE16B10429F7C4
:1057C00073945710E0CF8FEFC81AD80AE8E0CE16CE
:1057D000D10479F6DF91CF911F910F91FF90EF9057
:1057E000DF90CF90BF90AF909F908F907F905F9011
:1057F0004F903F902F900895A0E0B0E0E2E0FCE2EF
:105800000C94CD346C015B01342E4901380186E0E3
:10581000489F20011124F701E490EF012196EE202A
:1058200059F083019401432DB501C6010E947D2BDF
:10583000C40CD51CFE01F0CFCDB7DEB7E1E10C946E
:10584000E934A0E0B0E0E7E2FCE20C94CD343C01A6
:105850006B01342E5901480186E0489F2001112434
:10586000E701E99084019501432DB601C3010E942F
:105870007D2B640C751C88818052803690F3CDB7E7
:10588000DEB7E1E10C94E934A0E0B0E0EAE4FCE248
:105890000C94CC34EC015B01D42E4901380186E034
:1058A000489F100111242701F201E1902F0183018B
:1058B00094014D2DB501CE010E947D2BC20DD31D4B
:1058C000CA94C110F1CFCDB7DEB7E2E10C94E83451
:1058D00090932806809327067093260660932506EA
:1058E0000895EF92FF920F931F93CF93C82F80914B
:1058F00025069091260679018A019B014C2FBC0157
:1059000080912706909128060E94FC2B8091250605
:10591000909126062CE0C29F800D911D112490933A
:10592000260680932506CF911F910F91FF90EF904F
:105930000895EF92FF920F931F93CF93C82F8091FA
:1059400025069091260679018A019B014C2FBC0106
:1059500080912706909128060E94212C809125068F
:10596000909126062CE0C29F800D911D11249093EA
:10597000260680932506CF911F910F91FF90EF90FF
:105980000895A0E0B0E0E7ECFCE20C94D234FC0116
:10599000EB015901261B370BDA01A81BB90B0E943A
:1059A0009B346B017C019501215031094150510913
:1059B000BE01CF010E943C29E801812C912C5401A9
:1059C0008C149D04AE04BF0461F0FE018591949196
:1059D0000E94D3288FEF881A980AA80AB80A22963C
:1059E000EFCFCDB7DEB7ECE00C94EE34E0912E06AD
:1059F000F0912F0681E090E09C0100902B0602C000
:105A0000220F331F0A94E2F7322F3095418134235D
:105A10003183E0912E06F0912F063281232B2283D1
:105A200038B1AC010090300602C0440F551F0A94F3
:105A3000E2F7242F2095232328B937B1AC01009039
:105A4000290602C0440F551F0A94E2F7242F20951F
:105A5000232327B938B1AC010090290602C0440FB6
:105A6000551F0A94E2F7242F2095232328B9E091AB
:105A70002C06F0912D0600902A0602C0880F991F6F
:105A80000A94E2F7809592818923828385E38A953F
:105A9000F1F70000089587E880937A0086EB91E0A3
:105AA0000E94743D8F3F31F18093290685EB91E090
:105AB0000E94743D80932B0682EB91E00E94743D1E
:105AC00080932A068FEA91E00E94743D809330060D
:105AD00083EB91E00E94823D90932F0680932E06E7
:105AE00080EB91E00E94823D90932D0680932C06DE
:105AF00081E0089580E0089548B181E090E09C0144
:105B00000090290602C0220F331F0A94E2F7242BCB
:105B100028B948B19C010090300602C0220F331F03
:105B20000A94E2F7242B28B9E0912E06F0912F0673
:105B30009C0100902B0602C0220F331F0A94E2F74B
:105B40003181232B218347B19C010090300602C094
:105B5000220F331F0A94E2F7242B27B947B19C0187
:105B60000090290602C0220F331F0A94E2F7242B6B
:105B700027B9E0912C06F0912D0600902A0602C06C
:105B8000880F991F0A94E2F79181892B81830895E8
:105B9000CF93DF93F8940E94F62CE0912E06F091BB
:105BA0002F06C081D0E000902B0602C0D595C79586
:105BB0000A94E2F7C170DD2781E0C8270E947C2D9E
:105BC00078948C2FDF91CF910895E0912E06F0917B
:105BD0002F0620912B0640913006882309F45BC0E4
:105BE00081E090E0BC0102C0660F771F2A95E2F7C2
:105BF0009B012095318132233183E0912E06F09173
:105C00002F0632812323228357B19C0101C0220F2A
:105C10004A95EAF7252B27B938B1AC010090300638
:105C200002C0440F551F0A94E2F7242F2095232326
:105C300028B937B1AC010090290602C0440F551FA6
:105C40000A94E2F7242F2095232327B938B1AC0119
:105C50000090290602C0440F551F0A94E2F7242F32
:105C60002095232328B9E0912C06F0912D06009071
:105C70002A0602C0880F991F0A94E2F79181982B97
:105C80009183E0912C06F0912D069281892B8283DD
:105C9000809129065AC081E090E0BC0102C0660FE5
:105CA000771F2A95E2F79B013181322B3183E091F6
:105CB0002E06F0912F06209532812323228337B1BF
:105CC000BC0102C0660F771F4A95E2F7262F209588
:105CD000232327B938B1AC010090300602C0440F2D
:105CE000551F0A94E2F7242F2095232328B947B1A2
:105CF0009C010090290602C0220F331F0A94E2F78C
:105D0000242B27B948B19C010090290602C0220F1C
:105D1000331F0A94E2F7242B28B9E0912C06F09166
:105D20002D0600902A0602C0880F991F0A94E2F7F8
:105D30008095918198239183E0912C06F0912D0616
:105D400092818923828380913006806480937C00D5
:105D500072E07A95F1F700C080917A0080648093B8
:105D60007A0080917A0086FDFCCF80917800909136
:105D700079000895A8E0B0E0E0ECFEE20C94CC34A9
:105D8000F8944090530150905401612C712C89EB90
:105D900091E00E94823D8C018DEB91E00E94823D5A
:105DA0006C01E12CF12C80E00E94E52D98878F8317
:105DB0008090510190905201940140E050E029837D
:105DC0003A834B835C8387EB91E00E94823D9E8304
:105DD0008D838BEB91E00E94823D4C01A12CB12C74
:105DE00081E00E94E52D1C010E947C2D78944F815A
:105DF0005885CA01A0E0B0E09C01AD012C193D0915
:105E00004E095F09C301B2010E94103420E030E066
:105E1000A90198012C193D094E095F090E947634A9
:105E20006901C101A0E0B0E09C01AD012819390968
:105E30004A095B0969817A818B819C810E941034B7
:105E4000AD81BE818D0120E030E0A90198012819C3
:105E500039094A095B090E9476347901C701B60104
:105E60002896E2E10C94E8340F931F93CF93DF93CD
:105E7000F89480E00E94E52D8C0181E00E94E52DE0
:105E8000EC010E947C2D7894B801CE01DF91CF9176
:105E90001F910F910895CF92DF92EF92FF92CF93CF
:105EA000DF9320E330E040E050E0BA0180E00E9460
:105EB000981A8091B404813409F05EC08091B504D1
:105EC000843509F059C08091B604883309F054C074
:105ED0008091B704883509F04FC08091B804909143
:105EE000B904019709F048C08091BA049091BB04AD
:105EF000019709F041C08091C604813011F092E110
:105F000001C09AE190933506823019F080E890E064
:105F100002C080E091E09093340680933306C090F5
:105F2000D004D090D104E090D204F090D304C7E321
:105F3000D6E020E230E0B701A60180E00E94981A86
:105F4000892B29F4809133069091340617C0C992A9
:105F5000D992E992F9928091B4049091B504A091FC
:105F6000B604B091B704C80ED91EEA1EFB1E86E027
:105F7000CF3DD807F1F6E6CF80E090E0DF91CF91FA
:105F8000FF90EF90DF90CF900895A0E1B0E0EBECB0
:105F9000FFE20C94CC34FB01588B4F870197988714
:105FA0008F8380913506282F30E03A8729878F81AB
:105FB0009885B9010E942C3401E0060F80E1AF857D
:105FC000B8898C93809133069091340691838083B5
:105FD0000E94F731EFE4F2E33197F1F700C00000DF
:105FE00080913606081761F1E02EE81AE7FCE1948B
:105FF000C12CD12C0E2C000CFF08CE14DF0498F419
:106000000E94F731882329F087EE91EC0197F1F790
:1060100004C0AFECB2E51197F1F700C00000BFEF8C
:10602000CB1ADB0AEACF0E94F731882349F0EFEF61
:10603000F3EF21E0E150F0402040E1F700C0000024
:10604000009336060E94F0316C0110E001501109F6
:10605000A801440F551F440F551F5E834D83FA015D
:10606000E95CF94F80809180A280B3808114910413
:10607000A104B10419F4E12CF12C92C120E230E02A
:10608000B501A40180E00E94981A8091BC0490E0C0
:106090000817190781F72090BE043090BF0421141F
:1060A000310449F38091C8049091C904A091CA04B5
:1060B000B091CB04880E991EAA1EBB1E28E030E0CA
:1060C000B501A40180E00E94981A8091B4049091D7
:1060D000B504A091B604B091B704880E991EAA1E0B
:1060E000BB1EC10123E0880F991F2A95E1F7A50186
:1060F0009401281B390B410951092B873C874D8797
:106100005E8734E03C8300E010E01B82812C912C00
:106110005401E12CF12C4B845C846D847E841A82C2
:10612000198228E030E0B301A20180E00E94981AB1
:10613000892B09F44EC02091B50424FD45C08F8100
:10614000988569857A850E942C348F5F9091B4047C
:1061500089133AC08091B6049091B704AC014C19F0
:106160005D090115110571F0141615061CF417FDD3
:1061700009C005C04115510539F117FF25C0401769
:10618000510714F5909332068093310622FD04C026
:10619000AF85B8892C9305C0822F8260EF85F8897E
:1061A0008083AF85B8898C9186FF03C0BB81BF5FB8
:1061B000BB838090B8049090B904A090BA04B090CA
:1061C000BB048A01E980FA80E8E04E0E511C611C94
:1061D000711C29813A812F5F3F4F3A832983221610
:1061E000330609F09ECFAF85B8898C91811114C018
:1061F00080913106909132069093B5058093B40555
:10620000EF85F88980818F7789838083FB81F11105
:1062100015C00FEF1FEF54C00E94F0319C0186544F
:106220009A498B3B45E6940708F0C9010E94DA3190
:106230005C8151505C8351116ECFDACFED81FE81CC
:10624000E95CF94F40805180628073808091C8047E
:106250009091C904A091CA04B091CB04480E591E74
:106260006A1E7B1E0FEF1FEF28E030E0B301A20192
:1062700080E00E94981A4091B4045091B504609156
:10628000B6047091B704411551056105710599F087
:106290008091B90490E0E816F90641F48091B804C1
:1062A000803121F40091BA041091BB04440E551EB4
:1062B000661E771ED9CFAF85B8898C918F7B8C9362
:1062C00081149104A104B104A1F02091330630910E
:1062D0003406ED81FE81E95CF94F40815181628194
:1062E0007381480D591D6A1D7B1D80E00E94981A1C
:1062F0007C018981882311F0E12CF12C17FF0AC061
:106300008091310690913206C816D906E0F0865485
:106310009A4919C0D801AC54BB4F5D0100E011E0AF
:106320002091330630913406C501845B9440821776
:10633000930730F70E945F37B8010E944034F5019F
:1063400081935F01EDCF9C012C193D098AEB95E605
:10635000B1010E942C34C20ED31EFBEBCF16F5E622
:10636000DF0620F02AEBC21A25E6D20ACB018C0DFB
:106370009D1D8B3B35E6930710F08A5B95460E9486
:10638000DA310E94F731882329F08FE39FE10197EA
:10639000F1F704C0AFE3BFE11197F1F700C00000CF
:1063A000EF85F889808180958083C7016096E2E15E
:1063B0000C94E8342091840030918500369527951F
:1063C0008217930718F4B19AB19BFECF20918400F5
:1063D000309185003695279528173907B8F3089529
:1063E000809184009091850096958795089580917D
:1063F0003F0183FB882780F908952091E1063091C1
:10640000E2063695279540E050E060E472E48FE0C4
:1064100090E00E945434C90101970E94131F08950F
:106420008F929F92AF92BF92EF92FF920F931F9322
:10643000CF93DF93EC014C01A12CB12CE091BE0570
:10644000F091BF0542895389648975898416950640
:10645000A606B70608F05CC04150510961097109F0
:1064600097E076956795579547959A95D1F74F5F41
:106470005F4F6F4F7F4F7F936F935F934F93CE012B
:10648000880F892F881F990B919501969F938F9361
:106490008FE299E09F938F9384EB94E09F938F9387
:1064A0000E948D3734EBE32E34E0F32E0AE812E538
:1064B00020EE3FEF42E064E870E083E290E00E946B
:1064C000212C20E830E0B501A40180E00E94981A58
:1064D000E4E3F5E02DB73EB7265F3F4F0FB6F894E3
:1064E0003EBF0FBE2DBF34E0E43BF30719F092919D
:1064F0009383F9CF87FD06C09AEF9093B6048093FB
:10650000360503C09CEF9093B604C80FD11D18C088
:1065100089E2E82E89E0F82E0AE812E520EE3FEF46
:1065200042E064E870E083E290E00E94FC2B83E8A4
:1065300090E00E9495058EEF8093B604C0E0D0E015
:1065400085E58093B4048093B50463E870E084EB40
:1065500094E00E94331F63E870E084EB94E00E94B3
:10656000041F0E942C1F8FEF95EA2EE0815090406F
:106570002040E1F700C00000CE01DF91CF911F91D4
:106580000F91FF90EF90BF90AF909F908F900895E4
:1065900028E030E040E050E0BA0180E00E94981A24
:1065A0009091B4048091B705963471F49091B5043C
:1065B000953551F49091B6049A3431F49091B70422
:1065C000993411F4826001C08D7F8093B70580916A
:1065D000B70582FF03C088EE93E002C088E592E031
:1065E0009093E2068093E1060E94FD311092E0064E
:1065F0001092DF060895A0E0B0E0E1E0F3E30C9430
:10660000D0346C014601A12CB12CE091BE05F09173
:10661000BF0582899389A489B58988169906AA0637
:10662000BB0608F045C028E030E0B501A40180E0D9
:106630000E94981AC091B804D091B9048091B40412
:106640008436B1F48091B504813671F58091B60439
:10665000843751F58091B704813631F58091DF069A
:106660009091E00601969093E0068093DF0620C0AB
:106670008236D1F48091B5048136B1F48091B604AC
:10668000853791F48091B704843671F48091B70511
:1066900082FDB8CF8091BA049091BB049093E2063A
:1066A0008093E1060E94FD312896CC0EDD1EAACF14
:1066B00084EB94E06090BA047090BB04C091B8047D
:1066C000D091B9047F926F92DF93CF932091E2062D
:1066D0002F932091E1062F9329E039E03F932F93E8
:1066E0009F938F930E948D3794EBE92E94E0F92EBF
:1066F0000AE812E520EE37E041E069E970E08FE05A
:1067000090E00E94212C8DB79EB70A960FB6F894A0
:106710009EBF0FBE8DBFC301009741F0EFE9FFE0C0
:106720003197F1F700C000000197F6CFE091BE0568
:10673000F091BF0582899389A489B5898816990645
:10674000AA06BB0608F064C08091E0068F93809192
:10675000DF068F938BEF98E09F938F9384EB94E009
:106760009F938F930E948D3784EBE82E84E0F82E60
:106770000AE812E520EE3FEF42E064E870E083E2D1
:1067800090E00E94212C8601085F1F4F0F900F9010
:106790000F900F900F900F90DD24D39480E091E044
:1067A000209731F1C130F1E0DF0720F05E01BA94AB
:1067B000EC0102C0A12CB12CA80160E070E09E01A8
:1067C00080E00E94981A080F191FBE0184EB94E024
:1067D0000E94331FDD2041F08091B6048E3F21F4EA
:1067E0001092E0061092DF06D12CCE01E501D8CF41
:1067F0008091DF069091E006892B61F48FEF93EC96
:10680000E9E081509040E040E1F700C0000002C0A4
:1068100000E010E0C801CDB7DEB7EEE00C94EC3438
:10682000DB018F939F930E94B934BF91AF91A29FD8
:10683000800D911DA39F900DB29F900D112408957E
:10684000991B79E004C0991F961708F0961B881FC2
:106850007A95C9F780950895AA1BBB1B51E107C023
:10686000AA1FBB1FA617B70710F0A61BB70B881FE0
:10687000991F5A95A9F780959095BC01CD0108956F
:1068800097FB072E16F4009407D077FD09D00E94DD
:106890002C3407FC05D03EF4909581959F4F0895C8
:1068A000709561957F4F0895A1E21A2EAA1BBB1B1C
:1068B000FD010DC0AA1FBB1FEE1FFF1FA217B307CC
:1068C000E407F50720F0A21BB30BE40BF50B661FE2
:1068D000771F881F991F1A9469F7609570958095A6
:1068E00090959B01AC01BD01CF010895052E97FB4A
:1068F0001EF400940E948D3457FD07D00E9454343A
:1069000007FC03D04EF40C948D345095409530958F
:1069100021953F4F4F4F5F4F08959095809570950B
:1069200061957F4F8F4F9F4F0895EE0FFF1F05908A
:10693000F491E02D09940E94A334332312F48A1BAE
:106940009B0B0C94B434A29FB001B39FC001A39FD2
:10695000700D811D1124911DB29F700D811D112498
:10696000911D08950E94A334B7FF0895821B930BD5
:1069700008950E94A334A59F900DB49F900DA49FED
:10698000800D911D11240895B7FF0C94B9340E9415
:10699000B934821B930B08952F923F924F925F92CE
:1069A0006F927F928F929F92AF92BF92CF92DF921F
:1069B000EF92FF920F931F93CF93DF93CDB7DEB784
:1069C000CA1BDB0B0FB6F894DEBF0FBECDBF099418
:1069D0002A88398848885F846E847D848C849B846F
:1069E000AA84B984C884DF80EE80FD800C811B817D
:1069F000AA81B981CE0FD11D0FB6F894DEBF0FBEAC
:106A0000CDBFED0108955058BB27AA270E941B3522
:106A10000C946C360E945E3638F00E94653620F089
:106A200039F49F3F19F426F40C945B360EF4E0958C
:106A3000E7FB0C945536E92F0E947D3658F3BA17C0
:106A4000620773078407950720F079F4A6F50C9484
:106A50009F360EF4E0950B2EBA2FA02D0B01B90135
:106A600090010C01CA01A0011124FF27591B99F0C4
:106A7000593F50F4503E68F11A16F040A22F232FD0
:106A8000342F4427585FF3CF469537952795A79520
:106A9000F0405395C9F77EF41F16BA0B620B730BC7
:106AA000840BBAF09150A1F0FF0FBB1F661F771F38
:106AB000881FC2F70EC0BA0F621F731F841F48F4ED
:106AC000879577956795B795F7959E3F08F0B0CF76
:106AD0009395880F08F09927EE0F9795879508955D
:106AE0000E9484350C946C360E94653658F00E94E2
:106AF0005E3640F029F45F3F29F00C945536511171
:106B00000C94A0360C945B360E947D3668F3992372
:106B1000B1F3552391F3951B550BBB27AA27621799
:106B20007307840738F09F5F5F4F220F331F441FA6
:106B3000AA1FA9F335D00E2E3AF0E0E832D09150DA
:106B40005040E695001CCAF72BD0FE2F29D0660FC7
:106B5000771F881FBB1F261737074807AB07B0E80A
:106B600009F0BB0B802DBF01FF2793585F4F3AF010
:106B70009E3F510578F00C9455360C94A0365F3F3B
:106B8000E4F3983ED4F3869577956795B795F79596
:106B90009F5FC9F7880F911D9695879597F908957E
:106BA000E1E0660F771F881FBB1F6217730784071A
:106BB000BA0720F0621B730B840BBA0BEE1F88F729
:106BC000E09508950E94E9356894B1110C94A036BF
:106BD00008950E94853688F09F5798F0B92F99271D
:106BE000B751B0F0E1F0660F771F881F991F1AF0B8
:106BF000BA95C9F714C0B13091F00E949F36B1E048
:106C000008950C949F36672F782F8827B85F39F046
:106C1000B93FCCF3869577956795B395D9F73EF450
:106C200090958095709561957F4F8F4F9F4F0895F8
:106C3000E89409C097FB3EF4909580957095619516
:106C40007F4F8F4F9F4F9923A9F0F92F96E9BB27CC
:106C50009395F695879577956795B795F111F8CF48
:106C6000FAF4BB0F11F460FF1BC06F5F7F4F8F4FB3
:106C70009F4F16C0882311F096E911C0772321F0A9
:106C80009EE8872F762F05C0662371F096E8862F41
:106C900070E060E02AF09A95660F771F881FDAF798
:106CA000880F9695879597F9089597F99F6780E8DB
:106CB00070E060E008959FEF80EC089500240A944E
:106CC0001616170618060906089500240A941216C7
:106CD0001306140605060895092E0394000C11F4FA
:106CE000882352F0BB0F40F4BF2B11F460FF04C0A7
:106CF0006F5F7F4F8F4F9F4F089557FD9058440F00
:106D0000551F59F05F3F71F04795880F97FB991F0A
:106D100061F09F3F79F087950895121613061406C7
:106D2000551FF2CF4695F1DF08C016161706180654
:106D3000991FF1CF86957105610508940895E8942F
:106D4000BB2766277727CB0197F908950E94B936AC
:106D50000C946C360E945E3638F00E94653620F046
:106D6000952311F00C9455360C945B3611240C9439
:106D7000A0360E947D3670F3959FC1F3950F50E0C9
:106D8000551F629FF001729FBB27F00DB11D639FDD
:106D9000AA27F00DB11DAA1F649F6627B00DA11D83
:106DA000661F829F2227B00DA11D621F739FB00D29
:106DB000A11D621F839FA00D611D221F749F332799
:106DC000A00D611D231F849F600D211D822F762F32
:106DD0006A2F11249F5750409AF0F1F088234AF00F
:106DE000EE0FFF1FBB1F661F771F881F915050407B
:106DF000A9F79E3F510580F00C9455360C94A036AF
:106E00005F3FE4F3983ED4F3869577956795B79501
:106E1000F795E7959F5FC1F7FE2B880F911D96951B
:106E2000879597F908958F929F92AF92BF92CF92D4
:106E3000DF92EF92FF92CF93DF93EC01688179812B
:106E40008A819B81611571058105910521F464E2B8
:106E500079ED8BE597E02DE133EF41E050E00E94C2
:106E6000763449015A019B01AC01A7EAB1E40E94C2
:106E7000B9346B017C01ACEEB4EFA50194010E9422
:106E8000C734DC01CB018C0D9D1DAE1DBF1DB7FFAE
:106E900003C00197A109B04888839983AA83BB8363
:106EA0009F77DF91CF91FF90EF90DF90CF90BF90D1
:106EB000AF909F908F9008950E941337089585E5B5
:106EC00091E00E9413370895A0E0B0E0809355014F
:106ED00090935601A0935701B09358010895FB0178
:106EE000DC014150504048F005900D920020C9F758
:106EF00001C01D9241505040E0F70895FB01DC01B4
:106F00004150504048F001900D920020C9F701C057
:106F10001D9241505040E0F70895AEE0B0E0E3E943
:106F2000F7E30C94DA340D891E898EE08C831A8382
:106F300009838FEF9FE79E838D83AE01475E5F4F8E
:106F40006F89788DCE0101960E94C837EF81F88550
:106F5000E00FF11F10822E96E4E00C94F634AEE0C0
:106F6000B0E0E5EBF7E30C94DC348DE08C838B89A7
:106F70009C899A838983AE01495E5F4F6D897E89C2
:106F8000CE0101960E94453B2E96E2E00C94F83427
:106F9000ABE0B0E0EEECF7E30C94CC346C017B0199
:106FA0008A01FC0117821682838181FFCCC1CE0148
:106FB00001963C01F6019381F70193FD859193FFC2
:106FC00081917F01882309F4BAC1853239F493FD98
:106FD000859193FF81917F01853229F4B60190E07C
:106FE0000E94BE3CE7CF912C212C312CFFE1F31500
:106FF000D8F08B3279F038F4803279F08332A1F412
:10700000232D20611DC08D3261F0803369F4232D62
:10701000216016C0832D8260382EE32DE4603E2E61
:107020002AC0F32DF8601DC037FC2DC020ED280FBD
:107030002A3040F08E32B9F436FC81C1232D206411
:10704000322E19C036FE06C08AE0989E200D11240B
:10705000922E11C0EAE02E9E200D1124222EF32D37
:10706000F0623F2E08C08C3621F4832D8068382EC4
:1070700002C0883641F4F70193FD859193FF819119
:107080007F018111B3CF982F9F7D9554933028F4C1
:107090000C5F1F4F9FE399830DC0833631F0833718
:1070A00071F0833509F059C021C0F80180818983CE
:1070B0000E5F1F4F88248394912C530113C0280125
:1070C000F2E04F0E511CF801A080B18036FE03C0E3
:1070D000692D70E002C06FEF7FEFC5010E94753C23
:1070E0004C018201F32DFF773F2E16C0280122E0CC
:1070F000420E511CF801A080B18036FE03C0692DFC
:1071000070E002C06FEF7FEFC5010E946A3C4C0146
:10711000F32DF0683F2E820133FC1BC0822D90E0DE
:1071200088169906B0F4B60180E290E00E94BE3C59
:107130002A94F4CFF50137FC859137FE81915F01E8
:10714000B60190E00E94BE3C21102A9421E0821AF0
:1071500091088114910471F7E8C0843611F08936E2
:1071600041F5F80137FE07C060817181828193810A
:107170000C5F1F4F08C060817181072E000C880BC7
:10718000990B0E5F1F4FF32DFF763F2E97FF09C01F
:1071900090958095709561957F4F8F4F9F4FF068C8
:1071A0003F2E2AE030E0A3010E94133D882E86186E
:1071B00045C0853731F4232D2F7EB22E2AE030E0F2
:1071C00025C0932D997FB92E8F36C1F018F48835DC
:1071D00079F0B5C0803719F0883721F0B0C0E92FB9
:1071E000E061BE2EB4FE0DC0FB2DF460BF2E09C0C1
:1071F00034FE0AC0292F2660B22E06C028E030E0F7
:1072000005C020E130E002C020E132E0F801B7FE25
:1072100007C060817181828193810C5F1F4F06C01E
:107220006081718180E090E00E5F1F4FA3010E949A
:10723000133D882E8618FB2DFF773F2E36FE0DC09E
:10724000232D2E7FA22E891458F434FE0BC032FC5D
:1072500009C0832D8E7EA82E05C0B82CA32C03C098
:10726000B82C01C0B92CA4FE0FC0FE01E80DF11D21
:107270008081803321F49A2D997EA92E09C0A2FE27
:1072800006C0B394B39404C08A2D867809F0B394F1
:10729000A3FC11C0A0FE06C0B21488F4280C922CE6
:1072A0009B180EC0B21460F4B60180E290E00E9418
:1072B000BE3CB394F7CFB21418F42B1802C0982C2C
:1072C000212CA4FE10C0B60180E390E00E94BE3CD9
:1072D000A2FE17C0A1FC03C088E790E002C088E5C9
:1072E00090E0B6010CC08A2D867859F0A1FE02C04C
:1072F0008BE201C080E2A7FC8DE2B60190E00E9423
:10730000BE3C891438F4B60180E390E00E94BE3C94
:107310009A94F7CF8A94F301E80DF11D8081B601AC
:1073200090E00E94BE3C8110F5CF222009F442CEAD
:10733000B60180E290E00E94BE3C2A94F6CFF601AE
:107340008681978102C08FEF9FEF2B96E2E10C942C
:10735000E83420FD09C0FC0123FD05C022FF02C066
:107360007383628351834083089544FD17C046FDB3
:1073700017C0AB01BC01DA01FB01AA0FBB1FEE1F56
:10738000FF1F1094D1F74A0F5B1F6E1F7F1FCB01A9
:10739000BA01660F771F881F991F09C033E001C02B
:1073A00034E0660F771F881F991F3150D1F7620FA5
:1073B000711D811D911D08950F931F93CF93DF932E
:1073C0008C01C8010E94803CEC0197FD08C00E941E
:1073D000563C892BB1F7B801CE010E94FA3CCE0190
:1073E000DF91CF911F910F9108958F929F92AF924D
:1073F000BF92EF92FF920F931F93CF93DF938C0175
:10740000D62F7A01B22E0E94803C9C0133272B326A
:10741000310531F02D32310561F48B2D8068B82EA5
:10742000D15011F480E068C0C8010E94803C97FDF3
:10743000F9CFCB2DCD7F2B2D207309F58033F9F4B7
:10744000AA24AA94AD0E09F443C0C8010E94803C4E
:1074500097FD3EC09C012F7D33272835310549F427
:10746000C264D250A9F1C8010E94803C97FF07C0B6
:107470002FC0B6FE02C0C26001C0C261DA2D812CED
:10748000912C540120ED280F283080F0C4FF04C057
:10749000B8010E94FA3C19C02A3040F0C6FFF8CF6C
:1074A0002F7D3FEE320F363098F727504C2FC50115
:1074B000B4010E94B5394B015C01C260D15059F052
:1074C000C8010E94803C97FFDDCFC1FD04C0AACF58
:1074D000812C912C5401C7FF08C0B094A0949094C3
:1074E0008094811C911CA11CB11C2C2FB501A401FE
:1074F000C7010E94A93981E0DF91CF911F910F91BF
:10750000FF90EF90BF90AF909F908F900895A0E272
:10751000B0E0EDE8FAE30C94CF345C01962E7A01EA
:10752000F9018E010F5F1F4F680180E2D8011D92A3
:107530008A95E9F7D50113968C9080E090E0612C54
:10754000712C30E061E070E083FC259183FE219195
:107550008F01522E211103C080E090E092C02E35A1
:1075600011F4009751F1432F50E0481759073CF4AC
:107570002D3559F12D3219F4772009F103C0772008
:1075800009F46AC0452D469546954695D601A40F47
:10759000B11D452D47708B0102C0000F111F4A9588
:1075A000E2F7A8015C91452B4C93651459F05614F1
:1075B00010F45394E7CF5A94E5CF31E004C0772418
:1075C000739401C0712C0196BFCF772019F08E8182
:1075D00080628E83311103C08824839417C0F60122
:1075E0009E012F5D3F4F8081809581932E173F072D
:1075F000D1F7F2CFE114F10429F0D7018C93F70110
:1076000031967F019A94812C9920F9F0C5010E944E
:10761000803C97FD18C0FC01FF2723E0F595E79516
:107620002A95E1F7EC0DFD1D208130E0AC0147709B
:10763000552702C0359527954A95E2F720FDDACF08
:10764000B5010E94FA3C811087CFE114F10411F0DA
:10765000D7011C92C80115C0422F46954695469504
:10766000D601A40FB11D422F47708B0102C0000F3D
:10767000111F4A95E2F7A8015C91452B4C93622EAD
:10768000A2CFA096EFE00C94EB34A0E0B0E0EBE4E6
:10769000FBE30C94CF346C01EB015A01FC0117821F
:1076A0001682512CF601E380FE01E3FC8591E3FE96
:1076B0008191182FEF01882309F4EEC090E00E9419
:1076C000563C892B21F0C6010E94DC39EBCF1532E4
:1076D00041F4FE01E3FC1591E3FE1191EF01153237
:1076E00081F4C6010E94803C97FDD4C0412F50E038
:1076F0009C01332724173507A9F2B6010E94FA3CF2
:10770000CBC01A3239F4E3FC1591E3FE1191EF017D
:1077100001E001C000E0F12C20ED210F2A3080F4BF
:1077200002606F2D70E080E090E040E20E94B53989
:10773000F62EFE01E3FC1591E3FE1191EF01ECCF73
:1077400001FF03C0F11003C0A7C0FF24FA9418364C
:1077500019F01C3651F010C0FE01E3FC1591E3FE58
:107760001191EF01183641F408600460FE01E3FC5A
:107770001591E3FE1191EF01112309F48DC0612FE2
:1077800070E088EE90E00E945F3C892B09F484C091
:1077900000FD07C0F50180809180C50102965C0163
:1077A00002C0812C912C1E3651F4F601468157817E
:1077B00060E070E0202FC4010E94A93973CF133616
:1077C000A9F401FD02C0FF24F394C6010E94803C8D
:1077D00097FD60C08114910429F0F4018083C401F5
:1077E00001964C01FA94F110F0CF50C01B3559F4BA
:1077F0009E01A4016F2DC6010E94873AEC01892BDE
:1078000009F044C03EC0C6010E94DC3997FD42C069
:107810001F3661F128F4143639F1193651F128C0B8
:10782000133771F0153701F123C08114910429F049
:10783000F4016082C40101964C01FA94FF2071F0BA
:10784000C6010E94803C3C0197FD08C00E94563C46
:10785000892B59F3B601C3010E94FA3C81149104AB
:10786000A9F0F401108212C0006203C0006101C0DF
:107870000064202FA4016F2DC6010E94F5398111EB
:1078800005C0F6018381807329F406C000FD0ACF8C
:10789000539408CF552019F0852D90E002C08FEF4A
:1078A0009FEFCDB7DEB7EFE00C94EB3491110C9461
:1078B000713D803219F089508550C8F70895FC0158
:1078C0000590061621F00020D9F7C00108953197E0
:1078D000CF010895FC010590615070400110D8F768
:1078E000809590958E0F9F1F0895FC016150704008
:1078F00001900110D8F7809590958E0F9F1F0895E5
:10790000CF93DF93EC012B8120FF33C026FF0AC009
:107910002F7B2B838E819F8101969F838E838A810B
:1079200090E029C022FF0FC0E881F9818081082EF4
:10793000000C990B009719F420622B831AC0319622
:10794000F983E8830EC0EA85FB85099597FF09C096
:107950002B81019611F080E201C080E1822B8B83A4
:1079600008C02E813F812F5F3F4F3F832E83992791
:1079700002C08FEF9FEFDF91CF9108950F931F9378
:10798000CF93DF93FB01238121FD03C08FEF9FEF96
:107990002CC022FF16C046815781248135814217B1
:1079A000530744F4A081B1819D012F5F3F4F318384
:1079B00020838C93268137812F5F3F4F3783268327
:1079C00014C08B01EC01FB010084F185E02D0995C9
:1079D000892BE1F6D80116968D919C911797019607
:1079E00017969C938E931697CE01DF91CF911F919E
:1079F0000F910895FB01238120FF12C026FD10C0C6
:107A00008F3F3FEF930761F082832F7D20642383B4
:107A1000268137812150310937832683992708959C
:107A20008FEF9FEF0895FA01AA27283051F12031F6
:107A300081F1E8946F936E7F6E5F7F4F8F4F9F4F02
:107A4000AF4FB1E03ED0B4E03CD0670F781F891F44
:107A50009A1FA11D680F791F8A1F911DA11D6A0F12
:107A6000711D811D911DA11D20D009F468943F91C5
:107A70002AE0269F11243019305D3193DEF6CF01C4
:107A80000895462F4770405D4193B3E00FD0C9F78A
:107A9000F6CF462F4F70405D4A3318F0495D31FDF7
:107AA0004052419302D0A9F7EACFB4E0A69597954A
:107AB000879577956795BA95C9F700976105710520
:107AC00008959B01AC010A2E06945795479537956A
:107AD0002795BA95C9F7620F731F841F951FA01DC4
:107AE0000895992788270895F999FECF92BD81BD01
:107AF000F89A992780B50895A6E1B0E044E050E0F7
:107B00000C94AE3DA8E1B0E042E050E00C94AE3DF4
:107B1000262FF999FECF92BD81BDF89A019700B446
:107B2000021639F01FBA20BD0FB6F894FA9AF99AE6
:107B30000FBE08950396272F0E94893D0E94883D1D
:107B4000252F0E94893D242F0C94893D0196272FD3
:107B50000E94893D0C94883DDC01CB01FC01F99920
:107B6000FECF06C0F2BDE1BDF89A319600B40D9289
:0C7B700041505040B8F70895F894FFCF42
:107B7C003C02FF2901A82526040AFD239A03074B82
:107B8C0024FA0208D324AA02043426960201010323
:107B9C0003030303030303030303030103030303AB
:107BAC000303030303030303030307F00040010172
:107BBC0005012F000000000000000000000000FF85
:107BCC00FF4001F00001000000537461727400501A
:107BDC006175736500547572626F00457869740045
:107BEC00526F74617465005363726F6C6C00426FFA
:107BFC006F744431003130353000426C616E6B0073
:107C0C0053617665496D005361766500546F700061
:107C1C0050726576004F4B004E657874004C617362
:107C2C00740044303A0044313A3C656D7074793ECE
:107C3C0020202020200044323A3C656D7074793E3F
:107C4C0020202020200044333A3C656D7074793E2E
:107C5C0020202020200044343A3C656D7074793E1D
:107C6C00202020202000546170653A004E6577007A
:087C7C003E3E3E004366670036
:00000001FF
